:100000000C94BB010C94C0320C94ED320C94E301BF
:100010000C94E3010C94E3010C94E3010C94E301D0
:100020000C94E3010C94E3010C94E3010C94CE06D0
:100030000C94E3010C94E3010C94E3010C94E301B0
:100040000C94CC310C94E3010C9444060C9480067F
:100050000C94E3010C94E3010C94E3010C94E30190
:100060000C94E3010C94E301084AD73B3BCE016EAC
:1000700084BCBFFDC12F3D6C74319ABD56833DDAFF
:100080003D00C77F11BED9E4BB4C3E916BAAAABE0E
:10009000000000803F05A84CCDB2D44EB93836A937
:1000A000020C50B9918688083CA6AAAA2ABE000074
:1000B00000803F0664EC1B3C04BC163E3BE5B93CAB
:1000C000C93C37C29E5A3D660498083EEA69AAAA0E
:1000D0003E000000803F2020BF0020BF00BF007C0A
:1000E0002020202020202020202020202020202010
:1000F00020202000C8202020202020202020202078
:1001000020C900C8202020202020202020202020BE
:10011000C97C00D820202020202020202020202042
:10012000D97C00C820202020202020202020202032
:10013000C97C00C820202020202020202020202032
:10014000C97C00207265766F00206172737369004C
:100150006D696E6F706F7364206C6962726570692F
:100160006C6F74002020202020BABBBCBDBE7C2058
:1001700020202020CACBCCCDCE7C00626F6F74696A
:100180006E672075703AEDF2F2F2F2F2F2F2F300DD
:1001900062617474657279207761726E696E67202E
:1001A0000074787069642076616C756573006261B3
:1001B000726F2074656D700074656D706469737022
:1001C00020006163746976652000706173736976DD
:1001D000650075617674616C6B2000736574757071
:1001E0002073637265656E7C7C7C0043686172205D
:1001F000446F6E650A00526561647920666F7220F3
:10020000466F6E740A0055706461746520436861BE
:10021000725365740000407A10F35A00A0724E18B1
:10022000090010A5D4E80000E87648170000E40BA8
:1002300054020000CA9A3B000000E1F5050000806E
:10024000969800000040420F000000A086010000C8
:1002500000102700000000E8030000000064000018
:100260000000000A00000000000100000000002C57
:1002700076D888DC674F0823DFC1DFAE59E1B1B71C
:1002800096E5E3E453C63AE651997696E8E6C284E9
:1002900026EB898C9B62ED407C6FFCEFBC9C9F4001
:1002A000F2BAA56FA5F490055A2AF75C936B6CF926
:1002B000676DC11BFCE0E40D47FEF520E6B500D0FC
:1002C000ED902E0300943577050080841E08000011
:1002D000204E0A000000C80C333333330F986E12DF
:1002E000831141EF8D2114893BE65516CFFEE6DBE5
:1002F00018D1844B381BF77C1D901DA4BBE424202F
:100300003284725E228100C9F124ECA1E53D276EA2
:10031000616E00696E660000000000240027002A5C
:100320000000000000250028002B00000000002332
:100330000026002900040404040404040402020248
:100340000202020303030303030102040810204016
:10035000800102040810200102040810200000009F
:100360000700020100000304060000000000000076
:1003700000004F04150811241FBECFEFD8E0DEBFE8
:10038000CDBF13E0A0E0B1E0E2E7F0E702C00590E6
:100390000D92AE3FB107D9F716E0AEEFB3E001C062
:1003A0001D92A53BB107E1F713E0C6E7D3E004C017
:1003B0002297FE010E943338C237D107C9F70E9445
:1003C000FC330C9437380C940000FA01AA2728302B
:1003D00051F1203181F1E8946F936E7F6E5F7F4F12
:1003E0008F4F9F4FAF4FB1E03ED0B4E03CD0670F8E
:1003F000781F891F9A1FA11D680F791F8A1F911DE1
:10040000A11D6A0F711D811D911DA11D20D009F430
:1004100068943F912AE0269F11243019305D319372
:10042000DEF6CF010895462F4770405D4193B3E05B
:100430000FD0C9F7F6CF462F4F70405D4A3318F002
:10044000495D31FD4052419302D0A9F7EACFB4E0B3
:10045000A6959795879577956795BA95C9F700976B
:100460006105710508959B01AC010A2E069457950C
:10047000479537952795BA95C9F7620F731F841F63
:10048000951FA01D0895283008F027E03327DA01D2
:10049000990F311D87FD916000966105710539F452
:1004A00032602E5F3D9330E32A95E1F708959F3F38
:1004B00030F080387105610509F03C5F3C5F3D9389
:1004C000913008F08068911DDF93CF931F930F93B5
:1004D000FF92EF92192F987F9695E92F9695969512
:1004E000E90FFF27E159FD4F99273327EE24FF2419
:1004F000A701E70105900894079428F4360FE71E3A
:10050000F81E491F511D660F771F881F991F0694FB
:10051000A1F70590079428F4E70EF81E491F561F0F
:10052000C11D770F881F991F661F0694A1F70590BC
:10053000079428F4F80E491F561FC71FD11D880FB6
:10054000991F661F771F0694A1F70590079420F462
:10055000490F561FC71FD81F990F661F771F881F87
:100560000694A9F784911095177041F0D695C79518
:1005700057954795F794E7941A95C1F7E5E1F2E0AE
:1005800068941590159135916591959105907FE24C
:100590007395E118F10A430B560BC90BD009C0F74C
:1005A000E10CF11E431F561FC91FD01D7EF470338E
:1005B00011F48A95E6CFE894015030F0080F0AF460
:1005C0000027021708F4202F2395022F7A3328F0F2
:1005D00079E37D932A95E9F710C07D932A9589F6F2
:1005E000069497956795379517951794E118F10A32
:1005F000430B560BC90BD00998F023957E91739548
:100600007A3308F070E37C932013B8F77E91706121
:100610007D9330F0839571E37D9370E32A95E1F744
:100620001124EF90FF900F911F91CF91DF919927A7
:1006300087FD90950895CF93DF93BC01823091059B
:1006400010F462E070E0A091B306B091B406ED0141
:1006500040E050E0E0E0F0E021C088819981861719
:10066000970769F48A819B81309719F0938382837D
:1006700004C09093B4068093B306FE0134C068179B
:10068000790738F44115510519F08417950708F4D6
:10069000AC01FE018A819B819C01E9012097E9F66A
:1006A00041155105A9F1CA01861B970B049708F45F
:1006B000BA01E0E0F0E02AC08D919C911197841777
:1006C0009507F9F46417750781F412968D919C9142
:1006D0001397309719F09383828304C09093B406E4
:1006E0008093B306FD0132964CC0CA01861B970B5E
:1006F000FD01E80FF91F6193719302978D939C930D
:1007000040C0FD01828193819C01D9011097A1F61F
:100710008091B1069091B206892B41F480919F029D
:100720009091A0029093B2068093B1064091A102ED
:100730005091A2024115510541F44DB75EB7809129
:100740009D0290919E02481B590B2091B106309159
:10075000B206CA01821B930B8617970780F0AB0184
:100760004E5F5F4F8417950750F0420F531F509311
:10077000B2064093B106F9016193719302C0E0E0C3
:10078000F0E0CF01DF91CF910895CF93DF930097F1
:1007900009F450C0EC0122971B821A82A091B30683
:1007A000B091B406109709F140E050E0AC17BD07D6
:1007B00008F1BB83AA83FE0121913191E20FF31F5F
:1007C000AE17BF0779F48D919C911197280F391FAF
:1007D0002E5F3F4F3983288312968D919C911397FA
:1007E0009B838A834115510571F4D093B406C0935D
:1007F000B30620C012968D919C911397AD0100977E
:1008000011F0DC01D3CFFA01D383C283219131915E
:10081000E20FF31FCE17DF0769F488819981280F53
:10082000391F2E5F3F4FFA01318320838A819B81DC
:1008300093838283DF91CF910895FC0105906150ED
:1008400070400110D8F7809590958E0F9F1F0895E6
:10085000FC016150704001900110D8F7809590958F
:100860008E0F9F1F08956EBD0DB407FEFDCF8EB590
:1008700008958DE061E00E941A338BE061E00E94F0
:100880001A338CE060E00E941A338AE061E00E9433
:100890001A331CBC80E58CBD8DB58EB508958EEFE6
:1008A00093E00E9439040895FC011382128288EEBD
:1008B00093E0A0E0B0E084839583A683B78384EBC4
:1008C00092E0918380830895FC018089803419F43B
:1008D00021E030E002C020E030E0C9010895FC01D1
:1008E000818990E00895FC01648745876687478782
:1008F000089580E090E0089580E090E0089580E021
:1009000090E008950895EF92FF921F93CF93DF93A5
:10091000162F7A0186E060E00E9459338EEF93E053
:1009200060E00E9433048EEF93E060E00E943304A5
:100930008EEF93E069E00E9433048EEF93E0612F25
:100940000E943304C0E0D0E0F701EC0FFD1F1081DE
:100950008EEF93E06AE00E9433048EEF93E06C2FF9
:100960000E9433048EEF93E06BE00E9433048EEF1D
:1009700093E0612F0E9433042196C633D10521F7FD
:100980008EEF93E068E00E9433048EEF93E060EA1C
:100990000E9433048EEF93E060EA0E94330485FDE9
:1009A000F9CF8EEF93E060E00E9433048EEF93E086
:1009B0006CE00E94330486E061E00E945933DF91CD
:1009C000CF911F91FF90EF9008951F93CF93DF93E6
:1009D000EC01162F86E060E00E9459338EEF93E021
:1009E00060E00E943304112319F0113059F404C05F
:1009F0008EEF93E0688904C068896C618EEF93E0A4
:100A00000E94330486E061E00E945933DF91CF9168
:100A10001F910895EF92FF920F931F938EE1489FCD
:100A200070011124E60EF11C86E060E00E9459334B
:100A30000EEF13E0C80165E00E943304C8016F2D7A
:100A40000E943304C80166E00E943304C8016E2D81
:100A50000E9433041F910F91FF90EF900895EF9241
:100A6000FF920F931F937C010EEF13E0C80167E024
:100A70000E943304C8016FEF0E94330486E061E0F6
:100A80000E945933F70187858F5F87871F910F91E8
:100A9000FF90EF900895EF92FF920F931F93FC0148
:100AA000E7848EE1E89E700111248685E80EF11C32
:100AB00086E060E00E9459330EEF13E0C80164E065
:100AC0000E943304C80163E00E943304C80165E05A
:100AD0000E943304C8016F2D0E943304C80166E0F0
:100AE0000E943304C8016E2D0E9433041F910F91A0
:100AF000FF90EF9008951F93CF93DF93EC01162F93
:100B00006C3731F40E942F05CE010E944B050AC0BC
:100B10008EEF93E067E00E9433048EEF93E0612F45
:100B20000E94330481E090E0DF91CF911F910895FE
:100B30000F931F9386E060E00E9459330EEF13E09D
:100B4000C80164E00E943304C80164E00E943304D9
:100B500086E061E00E9459331F910F9108951F9321
:100B6000CF93DF93EC01188A16E0198B81EA96E0A7
:100B700060E973E00E942C31813049F480E4888B75
:100B800088E0898B86E060E00E94593302C0188AB1
:100B9000198B86E060E00E945933DF91CF911F915D
:100BA00008950F931F93CF93DF93EC0186E061E0EC
:100BB0000E941A3382E060E00E941A3382E061E012
:100BC0000E945933CE010E94AF0586E060E00E948A
:100BD00059338EEF93E06CEE0E9433048EEF93E076
:100BE0006FEF0E943304182F8EEF93E060E00E94B5
:100BF0003304688962608EEF93E00E94330462E3FD
:100C000070E080E090E00E9422328EEF93E06CE68C
:100C10000E9433041F7E8EEF93E0612F0E94330405
:100C20008889803419F00DE010E002C000E110E086
:100C3000109200041092FF0317C06091FF0370919F
:100C40000004605F8EEF93E00E9433048EEF93E028
:100C500069E00E9433048091FF03909100040196A3
:100C6000909300048093FF038091FF039091000410
:100C70008017910714F3CE0161E00E94E504DF9133
:100C8000CF911F910F9108951F920F920FB60F925F
:100C900011242F933F934F938F939F93EF93FF9341
:100CA0004091C60020919006309191062F5F3F4FF2
:100CB000809194069091950628233923809192067D
:100CC000909193062817390779F0809190069091BA
:100CD0009106E0919606F0919706E80FF91F408380
:100CE0003093910620939006FF91EF919F918F9101
:100CF0004F913F912F910F900FBE0F901F9018951D
:100D00001F920F920FB60F9211242F933F938F9340
:100D10009F93EF93FF9320919A0630919B068091C9
:100D200098069091990628173907E9F080919A065C
:100D300090919B06E0919E06F0919F06E80FF91FA7
:100D400080818093C60080919A0690919B060196BF
:100D500020919C0630919D068223932390939B06BD
:100D600080939A0610C02091980630919906809140
:100D70009A0690919B062817390729F48091C100A3
:100D80008F7D8093C100FF91EF919F918F913F9153
:100D90002F910F900FBE0F901F9018951F920F92DA
:100DA0000FB60F9211248F939F938091C10490915D
:100DB000C204892B51F08091C3049091C404019620
:100DC0009093C4048093C30409C08091C50490919A
:100DD000C60401969093C6048093C5049F918F9199
:100DE0000F900FBE0F901F901895CF93DF93482F51
:100DF000EB0180912606833009F45DC0843028F42D
:100E00008130C1F0823058F50AC0853009F4D2C073
:100E1000853008F4A8C0863009F0F2C0E9C04C3330
:100E200009F0EEC081E080932606488384EB80932E
:100E30002506E6C0842F90E0E0912506F0E0E82743
:100E4000F927EE53FD4F208120932506887F90706F
:100E5000809741F582E080932606498329C0242F9C
:100E600030E0E0912506F0E0E227F327EE53FD4F56
:100E7000808180932506809124068F5F80932406CD
:100E8000823018F43B832A83BBC0922F88272A81A3
:100E90003B81820F931F9B838A830A978F3F910523
:100EA00021F018F010922606ABC083E0809326064E
:100EB00010922406A5C0E42FF0E08091250690E072
:100EC000E827F927EE53FD4F808180932506609136
:100ED00024066F5F60932406623089F0633020F44B
:100EE000613009F08DC006C0633091F0643009F0C4
:100EF00087C022C0842F90E0A0E0B0E018C0242F6B
:100F000030E040E050E0542F432F322F222707C01B
:100F1000242F30E040E050E0A901332722278C81C4
:100F20009D81AE81BF81820F931FA41FB51F8C834B
:100F30009D83AE83BF8364C0242F30E040E050E047
:100F4000522F4427332722278C819D81AE81BF8178
:100F5000820F931FA41FB51F8C839D83AE83BF8315
:100F600060932606A5CF242F30E0E0912506F0E01F
:100F7000E227F327EE53FD4F808180932506809171
:100F800024068F5F80932406813019F08230C1F5EA
:100F900003C03987288734C0922F88272885398550
:100FA000280F391F398728878A819B810A97F1F09A
:100FB00085E07CCFE42FF0E08091250690E0E827E3
:100FC000F927EE53FD4F808180932506209124065A
:100FD0002F5F2093240630E0FB01E20FF31F4187CF
:100FE0008A819B810A972817390750F086E05ECFE7
:100FF000C75FDE4F4883C950D14087E08093260603
:1010000080912606873069F410922606C75FDE4F6E
:10101000909125068881C950D140981711F48A8192
:1010200001C080E0DF91CF9108958F92AF92CF926F
:10103000EF92FF920F931F9387E894E060E045ECF6
:1010400050E024EC30E000EC10E0B1ECEB2EF12CA1
:10105000CC24C394A8E9AA2EF0E28F2E0E949C2AE9
:1010600084EA94E00E9454041092B7041092B804E9
:101070001092B9041092BA041092BB041092BC04EE
:101080001092BD041092BE041092C0041092BF04CE
:101090001092B6041F910F91FF90EF90CF90AF90F8
:1010A0008F900895AF92BF92CF92DF92EF92FF920E
:1010B0000F931F93E0908C06F0908D0600918E06A2
:1010C00010918F068FE590E0A0E0B0E0E80EF91EE9
:1010D0000A1F1B1F0E9414326E157F05800791079F
:1010E00008F44EC0A090EC04B090ED04C090EE0463
:1010F000D090EF04C601B50120E030E040E85FE3A6
:101100000E949C36181694F5E0904406F09045062F
:1011100000914606109147060E94143220918C06D9
:1011200030918D0640918E0650918F06621B730B95
:10113000840B950B0E9472359B01AC01C601B50171
:101140000E94A73620E030E04AE754E40E94D934F8
:101150009B01AC01C801B7010E940C3460934406A6
:101160007093450680934606909347060E9414327A
:1011700060938C0670938D0680938E0690938F06F5
:101180001F910F91FF90EF90DF90CF90BF90AF90A5
:101190000895DF93CF9300D000D0CDB7DEB7FB0129
:1011A000E80FF91F628583859485258569838A8385
:1011B0009B832C83492F5C81782FCA010F900F905D
:1011C0000F900F90CF91DF910895AF92BF92DF9271
:1011D000EF92FF920F931F93CF93DF938C01809137
:1011E000270680FDE4C0F801F08087E894E06F2DC9
:1011F0000E947D2BE801C75FDE4FEF2DF0E0EE533C
:10120000FD4F80818883F801F18087E894E06F2D9D
:101210000E947D2BEF2DF0E0888190E0E827F927F0
:10122000EE53FD4F80818883F801F28087E894E0D7
:101230006F2D0E947D2BEF2DF0E0888190E0E82754
:10124000F927EE53FD4F80818883F801F38087E80A
:1012500094E06F2D0E947D2BEF2DF0E0888190E0CF
:10126000E827F927EE53FD4F80818883F801F48049
:1012700087E894E06F2D0E947D2BEF2DF0E08881B0
:1012800090E0E827F927EE53FD4F80818883F8012D
:101290002481358146815781232F342F452F5527AF
:1012A000F22E87E894E0622F0E947D2BEF2DF0E074
:1012B000888190E0E827F927EE53FD4F80818883ED
:1012C000F80124813581468157819A0144275527A9
:1012D000F22E87E894E0622F0E947D2BEF2DF0E044
:1012E000888190E0E827F927EE53FD4F80818883BD
:1012F000F8012481358146815781252F33274427E2
:101300005527F22E87E894E0622F0E947D2BEF2D67
:10131000F0E0888190E0E827F927EE53FD4F8081C7
:10132000888387E894E060E00E947D2BE881F0E00C
:10133000EE53FD4F8081888387E894E060E00E944F
:101340007D2BE881F0E0EE53FD4F80818883F8012A
:10135000828193810B9718F18AE0A82EB12CA00E00
:10136000B11E750112C0F701D1907F0187E894E0AA
:101370006D2D0E947D2BED2DF0E0888190E0E82717
:10138000F927EE53FD4F808188832E2D2A1930E0F6
:10139000F801828193810A972817390720F3075FA4
:1013A0001E4F87E894E0F80160810E947D2BDF9159
:1013B000CF911F910F91FF90EF90DF90BF90AF9072
:1013C0000895DF93CF93CDB7DEB7CA50D1400FB6A3
:1013D000F894DEBF0FBECDBF2CE329836A832AE0D9
:1013E00030E03C832B83FC0184819581A681B78109
:1013F0008D839E83AF83B887CE0101960E94E50856
:10140000C65FDE4F0FB6F894DEBF0FBECDBFCF91E3
:10141000DF91089581EA96E06AE773E00E942C313B
:10142000882331F586E696E6A6E6B0E480932906A1
:1014300090932A06A0932B06B0932C0680E090E0B0
:10144000A0E8BFE380932D0690932E06A0932F066D
:10145000B093300688EE93E0909332068093310685
:1014600081E8809333068DE8809334068DEF25C0A4
:1014700082E598EBAEE0B0E48093290690932A06CB
:10148000A0932B06B0932C0685E89BEEA1E5B0E473
:1014900080932D0690932E06A0932F06B0933006CE
:1014A00080EA94E190933206809331068BEF80932B
:1014B000330686E6809334068AEF809335060895D6
:1014C000FF920F931F9301EA16E0C8016CE773E0E7
:1014D0000E942C3180937006C8016EE773E00E9471
:1014E0002C3180937106C80160E873E00E942C31B2
:1014F00080935006C8016EE873E00E942C318093FF
:101500006806C8016AE873E00E942C318093660681
:10151000C80164E873E00E942C3180937206C80110
:1015200066E873E00E942C3180937306C8016CE872
:1015300073E00E942C3180935806C80162E973E081
:101540000E942C3180937406C80164E973E00E9404
:101550002C3180935706C80164EF73E00E942C3150
:10156000F82EC80165EF73E00E942C31382F20E07F
:101570002F0D311D3093760620937506C80166EF56
:1015800073E00E942C31F82EC80167EF73E00E94CF
:101590002C31382F20E02F0D311D30937806209309
:1015A0007706C80168EF73E00E942C31F82EC8015D
:1015B00069EF73E00E942C31382F20E02F0D311D90
:1015C00030937A0620937906C8016BEF73E00E948E
:1015D0002C3180934F061F910F91FF900895BC010D
:1015E00081EA96E00E942C3108956091D6047091B2
:1015F000D7048091D8049091D90420E030E040E1F4
:1016000052E40E94A73620E030E044EB53E40E940D
:10161000D9340E940A370E9441359B012550304041
:1016200037FF03C09B01215E3F4FA8E3B6E0F901FD
:10163000EE53FC4F80818C932F5F3F4F2432310556
:1016400014F020E030E0119686E0A334B80779F773
:101650001C9208952F923F924F925F926F927F92C9
:101660008F929F92AF92BF92CF92DF92EF92FF92B2
:101670000F931F93DF93CF9300D000D000D0CDB74E
:10168000DEB7182F662E2091CC043091CD042A3578
:10169000310530F0C9018D549F4F89359105E8F42B
:1016A00037FF02C02D543F4FC90137FF03C090954B
:1016B00081959F4F8A3191053CF0F4E48F2E912C57
:1016C000E9ED2E2E312C1DC00A975CF17BE3872EAD
:1016D000912C62ED262E312C20C02B35310514F0D3
:1016E000235B3040C90137FF03C0909581959F4F20
:1016F0008A31910554F056E5852E912C4CED242E1F
:10170000312C37E0A32EB12C15C00A9754F02DE4EC
:10171000822E912C94ED292E312C88E0A82EB12C0C
:1017200009C005E0802E912CB8E32B2E312CA9E0C6
:10173000AA2EB12C6091CE047091CF04882777FD3A
:101740008095982F0E94743527EA32E94BE25CEBD2
:101750000E94A7360E947B3720E030E040EA50E448
:101760000E94A73620E030E040E951E40E94A7360D
:101770000E940A3720E030E044E352E40E940C3437
:101780000E944135712EFEEBCF2EFFEFDF2E9B0125
:10179000442737FD4095542F29833A834B835C833C
:1017A000E4EA4E2EE4E05E2E4AEF5FEF240E351E93
:1017B0006091CC047091CD04882777FD8095982F97
:1017C0000E94743525E33AEF4EE85CE30E94A736A9
:1017D0000E947B377B018C01B601882777FD8095BD
:1017E000982F0E9474359B01AC01C801B7010E947B
:1017F000A7367B018C0169817A818B819C810E9453
:1018000074359B01AC01C801B7010E940C340E94E1
:1018100041359B01CB0101978A35910508F071C0D4
:1018200062E170E00E94E1378B012F5F3F4FAEEE27
:10183000BFEF6A9FC0016B9F900D7A9F900D11249E
:10184000820F931F62E070E00E94E1376D837E8318
:10185000E62CE01A4E2D4C5F84EA94E0672D0E943E
:101860000A0500D000D000D0EDB7FEB73196ADB775
:10187000BEB712965C924E92119720E031E033830E
:1018800022838D819E81880D991D958384830E947A
:101890007B2A4DB75EB74A5F5F4F0FB6F8945EBFC5
:1018A0000FBE4DBF8D819E818A159B0554F104307A
:1018B00011053CF593E0E90EC201672D4E2D0E9403
:1018C0000A0500D000D000D0EDB7FEB73196ADB715
:1018D000BEB712965C924E92119720E031E03383AE
:1018E00022834D815E81420D531D558344830E94A6
:1018F0007B2A8DB79EB706960FB6F8949EBF0FBE93
:101900008DBFACE0B0E0CA0EDB1E7394BEE4CB1614
:10191000D10409F04DCF26960FB6F894DEBF0FBE66
:10192000CDBFCF91DF911F910F91FF90EF90DF908E
:10193000CF90BF90AF909F908F907F906F905F906F
:101940004F903F902F900895823010F422E002C013
:10195000282F220F30E08DB79EB708970FB6F89466
:101960009EBF0FBE8DBFEDB7FEB7319684EA94E0FF
:10197000ADB7BEB712969C938E93119783E091E01A
:101980009383828322573F4F358324832F5F3F4FBA
:10199000378326830E947B2A8DB79EB708960FB6A1
:1019A000F8949EBF0FBE8DBF0895CF93DF93AC0117
:1019B000E091DE04F091DF04209136063091370685
:1019C000C9018C599F4F8E179F071CF4EA0121977C
:1019D00009C024563040E217F30714F0EA0102C0B0
:1019E000EA012196842F90E0C817D90729F081EAEF
:1019F00096E04C2F0E943331CE01DF91CF910895B4
:101A00000F931F9301EA16E0C80163EF73E041E012
:101A10000E943331C80164EF73E043E10E94333127
:101A2000C80165EF73E046E00E943331C80166EFFC
:101A300073E040E10E943331C80167EF73E047E291
:101A40000E943331C80168EF73E048E80E943331E7
:101A5000C80169EF73E043E10E9433311F910F9198
:101A60000895CF92DF92EF92FF920F931F937C0124
:101A7000D62EC72E04EA14E0C8016E2D4D2D0E940B
:101A80007304C8010E944B0500D000D0EDB7FEB72B
:101A90001283018383E391E0948383830E946A2A03
:101AA000EDB7FEB71283018383E291E094838383D1
:101AB0000E946A2AEDB7FEB71283018383E191E0A9
:101AC000948383830E946A2AEDB7FEB71283018351
:101AD00083E091E0948383830E946A2AEDB7FEB786
:101AE0001283018384EF90E0948383830E946A2AA7
:101AF0000F900F900F900F90C8010E942F05C70103
:101B000001966D2D7C2D0E942A0B1F910F91FF9045
:101B1000EF90DF90CF900895CF92DF92EF92FF92F7
:101B20000F931F93CF93DF93182F062F0E94143229
:101B300028EE33E040E050E00E94F43769017A017A
:101B4000C4EAD4E0CE01612F402F0E947304CE017D
:101B50000E944B058091FE049091FF04892B09F4AB
:101B600053C000910005109101058DB79EB74497B1
:101B70000FB6F8949EBF0FBE8DBFEDB7FEB731967E
:101B8000ADB7BEB71296DC93CE93119788E091E083
:101B90009383828383EB90E095838483C6016CE317
:101BA00070E00E94E137CB016CE370E00E94E13706
:101BB000978386832AE330E031872087C6016CE370
:101BC00070E00E94E1379387828785E690E09587F1
:101BD0008487C8016CE370E00E94CD37CB016CE3D1
:101BE00070E00E94E13797878687318B208BC80190
:101BF0006CE370E00E94CD37938B828B0E947B2A2E
:101C00008DB79EB7449633C0ADB7BEB71C970FB61D
:101C1000F894BEBF0FBEADBFEDB7FEB731961296BA
:101C2000DC93CE93119780E291E09383828383EBE0
:101C300090E095838483C6016CE370E00E94E137F5
:101C4000CB016CE370E00E94E137978386838AE3DF
:101C500090E091878087C6016CE370E00E94E137D5
:101C6000938782870E947B2A8DB79EB70C960FB60A
:101C7000F8949EBF0FBE8DBF84EA94E00E942F05AA
:101C8000DF91CF911F910F91FF90EF90DF90CF9058
:101C90000895EF92FF920F931F93282F462FA4EAE7
:101CA000EA2EA4E0FA2EC701622F0E947304C70136
:101CB0000E944B058DB79EB70A970FB6F8949EBF4A
:101CC0000FBE8DBF0DB71EB70F5F1F4FEDB7FEB72D
:101CD000F282E1828CE291E0F80193838283609149
:101CE00002057091030580910405909105052091EE
:101CF0002D0630912E0640912F06509130060E94FD
:101D0000A736F801648375838683978380EB90E020
:101D1000918780870E947B2A8DB79EB70A960FB65F
:101D2000F8949EBF0FBE8DBFC7010E942F051F9163
:101D30000F91FF90EF9008958F929F92AF92BF9274
:101D4000CF92DF92EF92FF920F931F93E82EF62E21
:101D500004EA14E0C8016E2D4F2D0E947304C801DF
:101D60000E944B058DB79EB70C970FB6F8949EBF97
:101D70000FBE8DBFEDB7FEB73196ADB7BEB71296A9
:101D80001C930E93119794E3892E91E0992E9382E0
:101D900082828DEEA82EB12CB582A48280910B0593
:101DA00090910C05A0910D05B0910E058683978347
:101DB000A087B187B3EFCB2ED12CD386C2860E94E9
:101DC0007B2A8DB79EB70C960FB6F8949EBF0FBEB8
:101DD0008DBFC8010E942F05F394C8016E2D4F2DB1
:101DE0000E947304C8010E944B05ADB7BEB71C9793
:101DF0000FB6F894BEBF0FBEADBFEDB7FEB73196BC
:101E000012961C930E93119793828282B582A482BC
:101E100080910F0590911005A0911105B0911205C8
:101E200086839783A087B187D386C2860E947B2A48
:101E30008DB79EB70C960FB6F8949EBF0FBE8DBFA0
:101E4000C8010E942F05F394C8016E2D4F2D0E94EA
:101E50007304C8010E944B05ADB7BEB71C970FB6FF
:101E6000F894BEBF0FBEADBFEDB7FEB73196129668
:101E70001C930E93119793828282B582A4828091E3
:101E8000130590911405A0911505B0911605868350
:101E90009783A087B187D386C2860E947B2A8DB79D
:101EA0009EB70C960FB6F8949EBF0FBE8DBFC801AB
:101EB0000E942F051F910F91FF90EF90DF90CF9020
:101EC000BF90AF909F908F9008950F931F93282FEE
:101ED000462F04EA14E0C801622F0E947304C8016F
:101EE0000E944B058DB79EB70A970FB6F8949EBF18
:101EF0000FBE8DBFEDB7FEB73196ADB7BEB7129628
:101F00001C930E9311978EE391E09383828389EB68
:101F100090E0958384838091FE049091FF049783E1
:101F2000868382E890E0918780870E947B2A8DB724
:101F30009EB70A960FB6F8949EBF0FBE8DBFC8011C
:101F40000E942F051F910F910895EF92FF920F931A
:101F50001F93282F462F34EAE32E34E0F32EC701D7
:101F6000622F0E947304C7010E944B058DB79EB774
:101F70000C970FB6F8949EBF0FBE8DBF0DB71EB75E
:101F80000F5F1F4FEDB7FEB7F282E18286E491E06A
:101F9000F8019383828384EE90E09583848360913B
:101FA000FC047091FD04882777FD8095982F0E948E
:101FB00074352AE037ED43E25CE30E94A736F8016E
:101FC00066837783808791878FE890E09387828705
:101FD0000E947B2A8DB79EB70C960FB6F8949EBFD1
:101FE0000FBE8DBFC7010E942F051F910F91FF905B
:101FF000EF9008950F931F93282F462F04EA14E0C3
:10200000C801622F0E947304C8010E944B058DB75E
:102010009EB70C970FB6F8949EBF0FBE8DBFEDB75D
:10202000FEB73196ADB7BEB712961C930E931197BB
:1020300086E491E09383828382EE90E095838483AB
:102040008091F8049091F904A091FA04B091FB04F6
:1020500086839783A087B1878EE890E093878287F5
:102060000E947B2A8DB79EB70C960FB6F8949EBF40
:102070000FBE8DBFC8010E942F051F910F910895BB
:102080000F931F93282F462F84EA94E0622F0E941B
:10209000730484EA94E00E944B058091DB0488235A
:1020A00019F420E531E057C0813019F424E531E01E
:1020B00052C0823019F428E531E04DC0833019F464
:1020C0002CE531E048C0843019F420E631E043C00B
:1020D000853019F424E631E03EC0863019F428E654
:1020E00031E039C0873019F42CE631E034C0883053
:1020F00019F420E731E02FC0893019F424E731E0EA
:102100002AC08A3019F428E731E025C08B3019F451
:102110002CE731E020C08C3019F420E831E01BC0FE
:102120008D3019F424E831E016C08E3019F428E817
:1021300031E011C08F3019F42CE831E00CC080314F
:1021400019F420E931E007C0813119F024E931E0C8
:1021500002C025E931E08DB79EB708970FB6F89415
:102160009EBF0FBE8DBFEDB7FEB7319604EA14E0F7
:10217000ADB7BEB712961C930E93119789E991E003
:102180009383828380EE90E09583848337832683D4
:102190000E947B2A8DB79EB708960FB6F8949EBF13
:1021A0000FBE8DBFC8010E942F051F910F9108958A
:1021B0000F931F93282F462F04EA14E0C801622FC3
:1021C0000E947304C8010E944B058DB79EB70A9701
:1021D0000FB6F8949EBF0FBE8DBFEDB7FEB7319618
:1021E000ADB7BEB712961C930E9311978EE991E08E
:1021F0009383828387E890E0958384838091DC04D5
:102200009091DD049783868385E290E091878087B3
:102210000E947B2A8DB79EB70A960FB6F8949EBF90
:102220000FBE8DBFC8010E942F051F910F91089509
:102230000F931F93282F462F04EA14E0C801622F42
:102240000E947304C8010E944B058DB79EB70A9780
:102250000FB6F8949EBF0FBE8DBFEDB7FEB7319697
:10226000ADB7BEB712961C930E93119788EA91E012
:10227000938382838091CE049091CF04958384834D
:1022800080EB90E09783868381EB90E09187808755
:102290000E947B2A8DB79EB70A960FB6F8949EBF10
:1022A0000FBE8DBFC8010E942F051F910F91089589
:1022B0000F931F93282F462F04EA14E0C801622FC2
:1022C0000E947304C8010E944B058DB79EB70A9700
:1022D0000FB6F8949EBF0FBE8DBFEDB7FEB7319617
:1022E000ADB7BEB712961C930E93119788EA91E092
:1022F000938382838091CC049091CD0495838483D1
:1023000080EB90E09783868382EB90E091878087D3
:102310000E947B2A8DB79EB70A960FB6F8949EBF8F
:102320000FBE8DBFC8010E942F051F910F91089508
:102330000F931F93282F462F04EA14E0C801622F41
:102340000E947304C8010E944B058DB79EB70A977F
:102350000FB6F8949EBF0FBE8DBFEDB7FEB7319696
:10236000ADB7BEB712961C930E93119780EB91E018
:102370009383828381EE90E0958384838091AB0286
:102380009091AC029783868385E290E09187808765
:102390000E947B2A8DB79EB70A960FB6F8949EBF0F
:1023A0000FBE8DBFC8010E942F051F910F91089588
:1023B0000F931F93282F462F04EA14E0C801622FC1
:1023C0000E947304C8010E944B058DB79EB70C97FD
:1023D0000FB6F8949EBF0FBE8DBFEDB7FEB7319616
:1023E000ADB7BEB712961C930E93119788EB91E090
:1023F0009383828382EC91E09583848380ED90E0E7
:102400009783868388E396E09187808781ED90E0CB
:10241000938782870E947B2A8DB79EB70C960FB652
:10242000F8949EBF0FBE8DBFC8010E942F051F915B
:102430000F9108950F931F93282F462F04EA14E05D
:10244000C801622F0E947304C8010E944B058DB71A
:102450009EB70A970FB6F8949EBF0FBE8DBFEDB71B
:10246000FEB73196ADB7BEB712961C930E93119777
:1024700080ED91E0938382838091D6049091D7047C
:10248000A091D804B091D90484839583A683B7839F
:1024900080EB90E0918780870E947B2A8DB79EB762
:1024A0000A960FB6F8949EBF0FBE8DBFC8010E945A
:1024B0002F051F910F9108950F931F93282F462FDB
:1024C00004EA14E0C801622F0E947304C8010E944C
:1024D0004B058DB79EB70C970FB6F8949EBF0FBEF5
:1024E0008DBFEDB7FEB73196ADB7BEB712961C9350
:1024F0000E93119788ED91E09383828386E190E0BB
:10250000958384838091F0049091F104A091F2046A
:10251000B091F30486839783A087B18788E890E021
:10252000938782870E947B2A8DB79EB70C960FB641
:10253000F8949EBF0FBE8DBFC8010E942F051F914A
:102540000F910895CF92DF92EF92FF920F931F9316
:10255000CF93DF93282F462FC4EAD4E0CE01622F19
:102560000E947304CE010E944B0560914406709155
:102570004506809146069091470620912D063091A0
:102580002E0640912F06509130060E94A7366B010F
:102590007C0120E030E04AE754E40E949C361816A3
:1025A000D4F58DB79EB70C970FB6F8949EBF0FBEAB
:1025B0008DBF0DB71EB70F5F1F4FADB7BEB71296D9
:1025C000DC93CE93119786E491E0F80193838283A4
:1025D0008EEF90E09583848360913106709132068E
:1025E000882777FD8095982F0E9474359B01AC0158
:1025F000C701B6010E94D934D80116966D937D9318
:102600008D939C931997809135061A968C931A97FF
:102610001B961C9221C08DB79EB70C970FB6F894ED
:102620009EBF0FBE8DBFEDB7FEB73196ADB7BEB73B
:102630001296DC93CE93119782EE91E0938382837E
:102640008EEF90E095838483C682D782E086F18600
:1026500080913406828713860E947B2AEDB7FEB7ED
:102660003C960FB6F894FEBF0FBEEDBF84EA94E02F
:102670000E942F05DF91CF911F910F91FF90EF9056
:10268000DF90CF900895EF92FF920F931F93282F22
:10269000462F54EAE52E54E0F52EC701622F0E9422
:1026A0007304C7010E944B058DB79EB70C970FB6F8
:1026B000F8949EBF0FBE8DBF0DB71EB70F5F1F4FA3
:1026C000EDB7FEB7F282E18288ED91E0F8019383E5
:1026D000828389EE90E0958384836091EC0470910D
:1026E000ED048091EE049091EF0420912906309141
:1026F0002A0640912B0650912C060E94A736F8011D
:1027000066837783808791878091330682871386DB
:102710000E947B2A8DB79EB70C960FB6F8949EBF89
:102720000FBE8DBFC7010E942F051F910F91FF9013
:10273000EF900895EF92FF920F931F93282F462F4B
:1027400064EAE62E64E0F62EC701622F0E9473044D
:10275000C7010E944B058DB79EB70C970FB6F89432
:102760009EBF0FBE8DBF0DB71EB70F5F1F4FEDB7DA
:10277000FEB7F282E18288ED91E0F80193838283D3
:1027800088EE90E0958384836091F4047091F50461
:102790008091F6049091F7042091290630912A0641
:1027A00040912B0650912C060E94A736F8016683B3
:1027B00077838087918780913306828713860E9472
:1027C0007B2A8DB79EB70C960FB6F8949EBF0FBEAE
:1027D0008DBFC7010E942F051F910F91FF90EF90B1
:1027E0000895EF92FF920F931F93282F462F74EABC
:1027F000E72E74E0F72EC701622F0E947304C70111
:102800000E944B058DB79EB70C970FB6F8949EBFEC
:102810000FBE8DBF0DB71EB70F5F1F4FEDB7FEB7D1
:10282000F282E18282EE91E0F8019383828386EE68
:1028300090E0958384836091E8047091E90480912D
:10284000EA049091EB0420912D0630912E064091E0
:102850002F06509130060E94A736F80166837783D1
:102860008087918780913406828713860E947B2A15
:102870008DB79EB70C960FB6F8949EBF0FBE8DBF56
:10288000C7010E942F051F910F91FF90EF900895AF
:10289000EF92FF920F931F93282F462FE4EAEE2E1C
:1028A000E4E0FE2EC701622F0E947304C7010E945C
:1028B0004B058DB79EB70C970FB6F8949EBF0FBE11
:1028C0008DBF0DB71EB70F5F1F4FEDB7FEB7F2827A
:1028D000E18282EE91E0F8019383828387EE90E0BB
:1028E000958384836091060570910705882777FD9D
:1028F0008095982F0E94743520912D0630912E06D8
:1029000040912F06509130060E94A736F801668349
:1029100077838087918780913406828713860E940F
:102920007B2A8DB79EB70C960FB6F8949EBF0FBE4C
:102930008DBFC7010E942F051F910F91FF90EF904F
:1029400008950F931F93282F462F04EA14E0C8011F
:10295000622F0E947304C8010E944B0580914806B3
:102960000E94A40CC8010E942F051F910F91089589
:10297000EF92FF920F931F93282F462FF4EAEF2E2A
:10298000F4E0FF2EC701622F0E947304C7010E946A
:102990004B058DB79EB70C970FB6F8949EBF0FBE30
:1029A0008DBF0DB71EB70F5F1F4FEDB7FEB7F28299
:1029B000E18282EE91E0F801938382838FE190E0DF
:1029C000958384836091490670914A0680914B06F5
:1029D00090914C060E94743520912D0630912E0660
:1029E00040912F06509130060E94A736F801668369
:1029F00077838087918780913406828713860E942F
:102A00007B2A8DB79EB70C960FB6F8949EBF0FBE6B
:102A10008DBFC7010E942F051F910F91FF90EF906E
:102A200008950F931F93282F462F04EA14E0C8013E
:102A3000622F0E947304C8010E944B058DB79EB798
:102A400040970FB6F8949EBF0FBE8DBFEDB7FEB78F
:102A50003196ADB7BEB712961C930E9311978CEEBC
:102A600091E09383828383E890E0958384838091CF
:102A7000D2049091D304A091D404B091D50486835C
:102A80009783A087B18784E890E0938782878091BD
:102A9000E2049091E304A091E404B091E5048487FA
:102AA0009587A687B7870E947B2A8DB79EB74096E9
:102AB0000FB6F8949EBF0FBE8DBFC8010E942F05B0
:102AC0001F910F9108950F931F93282F462F84EA8B
:102AD00094E0622F0E94730484EA94E00E944B0504
:102AE0008091E704282F30E0823030F4A4E0220FF8
:102AF000331FAA95E1F702C02150304000D000D02A
:102B000000D0EDB7FEB7319604EA14E0ADB7BEB71A
:102B100012961C930E93119780E091E09383828329
:102B2000358324830E947B2A8DB79EB706960FB605
:102B3000F8949EBF0FBE8DBFC8010E942F051F9144
:102B40000F9108950F931F93282F462F04EA14E046
:102B5000C801622F0E947304C8010E944B058DB703
:102B60009EB708970FB6F8949EBF0FBE8DBFEDB706
:102B7000FEB73196ADB7BEB712961C930E93119760
:102B80008EEF91E0938382838FE090E0958384833E
:102B90008091E604868317820E947B2A8DB79EB7B8
:102BA00008960FB6F8949EBF0FBE8DBFC8010E9455
:102BB0002F051F910F9108950F931F9304EA14E0BE
:102BC000C80163E045E00E947304C8010E944B0500
:102BD00000D000D0EDB7FEB71283018384E691E008
:102BE000948383830E946A2AEDB7FEB71283018320
:102BF00080E591E0948383830E946A2AEDB7FEB753
:102C00001283018389E491E0948383830E946A2A7A
:102C1000EDB7FEB71283018383E491E0948383834D
:102C20000E946A2A0F900F900F900F90C8010E9487
:102C30002F051F910F9108950F931F93282F462F53
:102C400004EA14E0C801622F0E947304C8010E94C4
:102C50004B0500D000D0EDB7FEB7128301838BE7A0
:102C600091E0948383830E946A2A0F900F900F90C3
:102C70000F90C8010E942F051F910F910895EF92A8
:102C8000FF920F931F93CF93DF930E9414322091F2
:102C9000520630915306409154065091550626171E
:102CA00037074807590708F08AC10E9414326C5050
:102CB0007E4F8F4F9F4F60935206709353068093C1
:102CC00054069093550604EA14E0C8010E94980542
:102CD000C80165E043E00E947304C8010E944B05EF
:102CE00000D000D0EDB7FEB7128301838BED91E0E9
:102CF000948383830E946A2A0F900F900F900F9005
:102D00008091360690913706892B31F080914D06DF
:102D100090914E06892B81F48091DE049091DF041E
:102D200090933706809336068091E0049091E104F9
:102D300090934E0680934D062091E0043091E1047B
:102D400040914D0650914E06C90184569040481757
:102D5000590724F4809151068F5F08C02C593F4FCA
:102D6000241735072CF48091510681508093510629
:102D700080915106181614F081E003C084301CF0D5
:102D800083E08093510680915106823009F462C03D
:102D9000833009F4BEC0813009F00DC100D000D0ED
:102DA000C4EAD4E0EDB7FEB7D283C18382ED91E0EF
:102DB000948383830E946A2A809127060F900F9044
:102DC0000F900F9080FF22C000D000D0EDB7FEB76B
:102DD000D283C1838AEC91E0948383830E946A2A20
:102DE0008091360690913706845690400F900F9050
:102DF0000F900F902091DE043091DF0428173907DF
:102E00000CF0D9C0809127068E7F21C000D000D061
:102E1000EDB7FEB7D283C18382EC91E094838383C4
:102E20000E946A2A80913606909137068C599F4FEE
:102E30000F900F900F900F902091DE043091DF04DF
:102E4000821793070CF0B7C08091270681608093AA
:102E50002706B1C000D000D0C4EAD4E0EDB7FEB779
:102E6000D283C18388EB91E0948383830E946A2A92
:102E70000F900F900F900F9080914F06882301F1D3
:102E800000D000D0EDB7FEB7D283C1838EEA91E0C7
:102E9000948383830E946A2A809136069091370634
:102EA000845690400F900F900F900F902091DE0469
:102EB0003091DF04281739071CF510924F0620C007
:102EC00000D000D0EDB7FEB7D283C18381EA91E094
:102ED000948383830E946A2A8091360690913706F4
:102EE0008C599F4F0F900F900F900F902091DE0400
:102EF0003091DF04821793071CF481E080934F0622
:102F000081EA96E06BEF73E040914F060E94333107
:102F100052C000D000D0B4EAEB2EB4E0FB2EEDB7E7
:102F2000FEB7F282E18280E991E0948383830E947C
:102F30006A2A8DB79EB708970FB6F8949EBF0FBE4A
:102F40008DBF0DB71EB70F5F1F4FEDB7FEB7F282F3
:102F5000E18284E092E0F8019383828360915006DD
:102F600070E080E090E00E94723520E030E040E2C6
:102F700051E40E94D934F801648375838683978372
:102F800086E790E09187808780E290E09387828750
:102F90000E947B2A8DB79EB70C960FB6F8949EBF01
:102FA0000FBE8DBF8091500690E060E873E00E94F4
:102FB000D50C8093500684EA94E00E942F05DF919F
:102FC000CF911F910F91FF90EF900895BF92CF92F4
:102FD000DF92EF92FF920F931F93CF93DF93E82E30
:102FE000D62E0E94143220915F06309160064091E7
:102FF000610650916206261737074807590708F0FF
:1030000024C1809163068823C9F08093AD02109299
:1030100063068CE092E090936506809364060E94BC
:1030200014326C507E4F8F4F9F4F60935F067093AA
:1030300060068093610690936206C2C08091AD02E3
:10304000A82FB0E07091DA044091640650916506B3
:10305000F090C7041091E70400915606609118059E
:10306000E091AB02F091AC0280915706C82FD0E0FE
:10307000B0905806909117059D012F5F3F4F273064
:1030800031051CF021E030E019C02330310531F169
:103090002430310544F42130310581F022303105EE
:1030A00009F057C012C02530310591F125303105A6
:1030B000ECF02630310509F04CC037C0723008F012
:1030C00048C049E152E081E049C083E0C82EFC14C9
:1030D00009F43FC046E252E082E040C01230C8F539
:1030E0000023B9F143E352E083E038C0623088F155
:1030F000633039F0643041F0623041F440E452E032
:1031000005C04DE452E002C04AE552E084E026C02A
:10311000EC17FD07F4F48FEFED39F807D1F0BB2081
:10312000C1F447E652E085E019C0723090F4923065
:1031300080F0933039F0943041F0923051F444E70C
:1031400052E005C040E852E002C04DE852E086E09F
:1031500005C02A173B0709F090CF60C05093650661
:10316000409364068093630681E0809359060E9431
:10317000143268517C4F8F4F9F4F60935F0670935E
:10318000600680936106909362060E941432605636
:10319000704F8F4F9F4F60935B0670935C068093D8
:1031A0005D0690935E0680915A06882321F084EA9A
:1031B00094E00E94980510925A0602C01092590697
:1031C00004EA14E0C8016E2D4D2D0E947304C8015D
:1031D0000E944B0500D000D000D0EDB7FEB731966D
:1031E000ADB7BEB712961C930E9311978AE992E081
:1031F000938382838091640690916506958384838E
:103200000E947B2A8DB79EB706960FB6F8949EBF94
:103210000FBE8DBFC8010E942F0517C050936506D1
:1032200040936406109263060E94143220915B065C
:1032300030915C0640915D0650915E062617370777
:103240004807590708F4BACFBBCFDF91CF911F9140
:103250000F91FF90EF90DF90CF90BF900895EF9285
:10326000FF920F931F9380916606843009F056C039
:103270009091DB04943008F027C180916F06891784
:10328000A1F190936F060E94143260936B067093C5
:103290006C0680936D0690936E0690916F068091F8
:1032A000AE02981711F580915A06813091F0813065
:1032B00018F08230B1F413C011E010935A060E9446
:1032C0001432615375478040904030F41093670684
:1032D00008C082E080935A061092670602C01092DE
:1032E0005A0684EA94E00E9498050E9414322091C4
:1032F0006B0630916C0640916D0650916E06621B14
:10330000730B840B950B615D77408040904008F40F
:10331000DBC08091DB048093AE02D6C0853029F4F7
:103320008091A3029091A40214C0863029F4809168
:10333000A5029091A6020DC0873029F48091A702C2
:103340009091A80206C0883041F48091A902909122
:10335000AA0290936A06809369068091680620917C
:10336000690630916A06882309F04AC0C90189506C
:1033700097408F5A9440C8F40E94143261537547A5
:103380008040904020F481E0809367060CC08091DB
:103390006706882341F480915906882321F484EA42
:1033A00094E00E94980582E028C044E0203B340766
:1033B00068F480915A06882349F01092670684EADF
:1033C00094E00E94980510925A067EC0205B34401B
:1033D0002955324008F078C080915A06813009F4AE
:1033E00073C080915906882309F06EC01092670659
:1033F00084EA94E00E94980581E080935A0664C0B4
:10340000215B344008F460C00E9414326153754758
:103410008040904008F041C0809167068823E9F51C
:10342000E0906B06F0906C0600916D0610916E06B0
:1034300088EE93E0A0E0B0E0E80EF91E0A1F1B1F23
:103440000E941432E616F70608071907E8F581E02E
:103450008093670617C01092670684EA94E00E9482
:10346000980580915A06823019F410925A0603C0CA
:103470008F5F80935A0680915A06823018F082E05E
:1034800080935A060E94143260936B0670936C0608
:1034900080936D0690936E0617C0E0906B06F090D7
:1034A0006C0600916D0610916E0688EE93E0A0E028
:1034B000B0E0E80EF91E0A1F1B1F0E941432E61628
:1034C000F7060807190738F21F910F91FF90EF9048
:1034D000089580916606843010F00E942F19809123
:1034E0006706882319F00E943F160895809107040B
:1034F00080FF08C060916D0480916B0490E070E0E3
:103500000E94E61780915A06823008F012C2A82F56
:10351000B0E0FD01EF5FFB4F808185FF0BC0FD0137
:10352000E35EFB4F6081A55EBB4F8C9190E070E045
:103530000E94A21580915A06A82FB0E0FD01EF5F0E
:10354000FB4F808186FF0BC0FD01EF5DFB4F60816B
:10355000A15EBB4F8C9190E070E00E94631580915A
:103560005606882309F43FC080915A06A82FB0E080
:10357000FD01EF5FFB4F808187FF0BC0FD01EB5D1D
:10358000FB4F6081AD5DBB4F8C9190E070E00E947D
:10359000111580915A06A82FB0E0FD01ED5FFB4F99
:1035A000808184FF0BC0FD01E35CFB4F6081A55C63
:1035B000BB4F8C9190E070E00E94B81480915A0645
:1035C000A82FB0E0FD01ED5FFB4F808183FF0BC0B2
:1035D000FD01E75CFB4F6081A95CBB4F8C9190E0E3
:1035E00070E00E94A11480915A06A82FB0E0FD015E
:1035F000EB5FFB4F808187FF0BC0FD01EB5AFB4F58
:103600006081AD5ABB4F8C9190E070E00E944814ED
:1036100080915A06A82FB0E0FD01E95FFB4F808141
:1036200083FF0BC0FD01EB58FB4F6081AD58BB4FD2
:103630008C9190E070E00E945C1280915A06A82F55
:10364000B0E0FD01EB5FFB4F808181FF0BC0FD010E
:10365000E35AFB4F6081A55ABB4F8C9190E070E01C
:103660000E949A1380915606882309F444C08091E1
:10367000E704823008F43FC080915A06A82FB0E0DA
:10368000FD01E75FFB4F808182FF0BC0FD01EF571B
:10369000FB4F6081A158BB4F8C9190E070E00E947D
:1036A000A21280915A06A82FB0E0FD01EB5FFB4FFC
:1036B000808182FF0BC0FD01EF5AFB4F6081A15B4F
:1036C000BB4F8C9190E070E00E94F11380915A06FC
:1036D000A82FB0E0FD01EB5FFB4F808183FF0BC0A3
:1036E000FD01E75AFB4F6081A95ABB4F8C9190E0D6
:1036F00070E00E94431380915A06A82FB0E0FD01AC
:10370000ED5FFB4F808181FF0BC0FD01EF5CFB4F44
:103710006081A15DBB4F8C9190E070E00E941A1215
:1037200080915A06A82FB0E0FD01ED5FFB4F80812C
:1037300080FF0BC0FD01E35DFB4F6081A55DBB4FCA
:103740008C9190E070E00E94D81180915A06A82FC9
:10375000B0E0FD01E95FFB4F808186FF0BC0FD01FA
:10376000E358FB4F6081A558BB4F8C9190E070E00F
:103770000E94981180915A06A82FB0E0FD01EF5FDA
:10378000FB4F808182FF0BC0FD01EB5EFB4F608130
:10379000AD5EBB4F8C9190E070E00E94581180911B
:1037A0005A06A82FB0E0FD01EF5FFB4F808181FF3B
:1037B0000BC0FD01EF5EFB4F6081A15FBB4F8C91A1
:1037C00090E070E00E94181180915A06A82FB0E096
:1037D000FD01EB5FFB4F808184FF0BC0FD01EF59C2
:1037E000FB4F6081A15ABB4F8C9190E070E00E942A
:1037F000D81080915A06A82FB0E0FD01EB5FFB4F77
:10380000808185FF0BC0FD01EB59FB4F6081AD59F5
:10381000BB4F8C9190E070E00E94401080915A065E
:10382000A82FB0E0FD01EF5FFB4F808183FF0BC04D
:10383000FD01E75EFB4F6081A95EBB4F8C9190E07C
:1038400070E00E94FA0F80915A06A82FB0E0FD01A7
:10385000EB5FFB4F808180FF0BC0FD01E35BFB4F03
:103860006081A55BBB4F8C9190E070E00E94A50F3A
:1038700080915A06A82FB0E0FD01EF5FFB4F8081D9
:1038800084FF0BC0FD01E75DFB4F6081A95DBB4F6D
:103890008C9190E070E00E94650F80915A06A82FED
:1038A000B0E0FD01E75FFB4F808181FF18C0809190
:1038B0004F06FD01ED57FB4F813049F4AB57BB4F2D
:1038C0006C91808190E070E00E94490E08C0AB5777
:1038D000BB4F6C91808190E070E00E949C0E8091C3
:1038E0005A06A82FB0E0FD01ED5FFB4F808187FFF6
:1038F0000BC0FD01E75BFB4F6081A95BBB4F8C9167
:1039000090E070E00E948C0D80915A06A82FB0E0E4
:10391000FD01EB5FFB4F808186FF0BC0FD01E75986
:10392000FB4F6081A959BB4F8C9190E070E00E94E1
:10393000310D089584EA94E00E9498050E94DC15F8
:103940000E940A0A0895CF93DF93EC0184EA94E081
:103950000E946F04C817D9073CF084EA94E00E94E3
:103960006404892B09F42397CE01DF91CF91089548
:10397000EF92FF920F931F93CF93DF9300915A061C
:1039800010E08AEF90E0089F7001099FF00C189FEB
:10399000F00C1124C7010E94EF0AF801EF5FFB4F02
:1039A000882319F08081816002C080818E7F8083AE
:1039B00080915A06C82FD0E0C70102960E94EF0AF4
:1039C000C55FDB4F888380915A06C82FD0E0C701BE
:1039D00004960E94EF0A90E00E94A31CC35FDB4F95
:1039E000888300915A0610E0C70188569F4F0E94B5
:1039F000EF0AF801EF5FFB4F882319F080818061A7
:103A000002C080818F7E808380915A06C82FD0E0CB
:103A1000C70186569F4F0E94EF0AC95DDB4F88831E
:103A200080915A06C82FD0E0C70184569F4F0E944C
:103A3000EF0A90E00E94A31CC75DDB4F88830091D2
:103A40005A0610E0C70106960E94EF0AF801EF5FE0
:103A5000FB4F882319F08081826002C080818D7FB6
:103A6000808380915A06C82FD0E0C70108960E9433
:103A7000EF0AC15FDB4F888380915A06C82FD0E0E0
:103A8000C7010A960E94EF0A90E00E94A31CCF5E35
:103A9000DB4F888300915A0610E0C7010C960E9404
:103AA000EF0AF801EF5FFB4F882319F080818460F3
:103AB00002C080818B7F808380915A06C82FD0E01E
:103AC000C7010E960E94EF0ACD5EDB4F888380917E
:103AD0005A06C82FD0E0C70140960E94EF0A90E036
:103AE0000E94A31CCB5EDB4F888300915A0610E036
:103AF000C70142960E94EF0AF801EF5FFB4F88234F
:103B000019F08081886002C08081877F80838091E6
:103B10005A06C82FD0E0C70144960E94EF0AC95E3A
:103B2000DB4F888380915A06C82FD0E0C7014696A4
:103B30000E94EF0A90E00E94A31CC75EDB4F8883BF
:103B400000915A0610E0C7014E960E94EF0AF80154
:103B5000EF5FFB4F882319F08081806202C0808173
:103B60008F7D808380915A06C82FD0E0C701809650
:103B70000E94EF0AC55EDB4F888380915A06C82FEA
:103B8000D0E0C70182960E94EF0A90E00E94A31C39
:103B9000C35EDB4F888300915A0610E0C70184960C
:103BA0000E94EF0AF801EF5FFB4F882319F0808134
:103BB000806402C080818F7B808380915A06C82FE9
:103BC000D0E0C70186960E94EF0AC15EDB4F888372
:103BD00080915A06C82FD0E0C70188960E94EF0A4C
:103BE00090E00E94A31CCF5DDB4F888300915A06B2
:103BF00010E0C7018A960E94EF0AF801EF5FFB4FC1
:103C0000882319F08081806802C080818F7780834B
:103C100080915A06C82FD0E0C7018C960E94EF0A07
:103C2000CD5DDB4F888380915A06C82FD0E0C70155
:103C30008E960E94EF0A90E00E94A31CCB5DDB4FA2
:103C4000888300915A0610E0C701C0960E94EF0ACF
:103C5000F801ED5FFB4F882319F08081816002C07D
:103C600080818E7F808380915A06C82FD0E0C70163
:103C7000C2960E94EF0AC55DDB4F888380915A0689
:103C8000C82FD0E0C701C4960E94EF0A90E00E94BE
:103C9000A31CC35DDB4F888300915A0610E0C70167
:103CA000C6960E94EF0AF801ED5FFB4F882319F0DA
:103CB0008081826002C080818D7F808380915A06DE
:103CC000C82FD0E0C701C8960E94EF0AC15DDB4F44
:103CD000888380915A06C82FD0E0C701CA960E94F7
:103CE000EF0A90E00E94A31CCF5CDB4F8883009119
:103CF0005A0610E0C701CC960E94EF0AF801ED5F6A
:103D0000FB4F882319F08081846002C080818B7F03
:103D1000808380915A06C82FD0E0C701CE960E94BA
:103D2000EF0ACD5CDB4F888380915A06C82FD0E024
:103D3000C701805C9F4F0E94EF0A90E00E94A31C85
:103D4000CB5CDB4F888300915A0610E0C701885B8B
:103D50009F4F0E94EF0AF801ED5FFB4F882319F097
:103D60008081806102C080818F7E808380915A062D
:103D7000C82FD0E0C701865B9F4F0E94EF0AC55C49
:103D8000DB4F888380915A06C82FD0E0C701845B3F
:103D90009F4F0E94EF0A90E00E94A31CC35CDB4F80
:103DA000888300915A0610E0C7018E5B9F4F0E94E6
:103DB000EF0AF801ED5FFB4F882319F080818860DE
:103DC00002C08081877F808380915A06C82FD0E00F
:103DD000C7018C5B9F4F0E94EF0AC95CDB4F888351
:103DE00080915A06C82FD0E0C7018A5B9F4F0E947E
:103DF000EF0A90E00E94A31CC75CDB4F8883009110
:103E00005A0610E0C701805B9F4F0E94EF0AF8013D
:103E1000ED5FFB4F882319F08081806202C08081B2
:103E20008F7D808380915A06C82FD0E0C7018E5ABB
:103E30009F4F0E94EF0AC15CDB4F888380915A0636
:103E4000C82FD0E0C7018C5A9F4F0E94EF0A90E024
:103E50000E94A31CCF5BDB4F888300915A0610E0C1
:103E6000C7018A5A9F4F0E94EF0AF801ED5FFB4F8E
:103E7000882319F08081806402C080818F7B8083D9
:103E800080915A06C82FD0E0C701885A9F4F0E94E0
:103E9000EF0ACD5BDB4F888380915A06C82FD0E0B4
:103EA000C701865A9F4F0E94EF0A90E00E94A31C10
:103EB000CB5BDB4F888300915A0610E0C701825626
:103EC0009F4F0E94EF0AF801ED5FFB4F882319F026
:103ED0008081806802C080818F77808380915A06BC
:103EE000C82FD0E0C70180569F4F0E94EF0AC95BE0
:103EF000DB4F888380915A06C82FD0E0C7018E55CA
:103F00009F4F0E94EF0A90E00E94A31CC75BDB4F0B
:103F1000888300915A0610E0C7018E599F4F0E9476
:103F2000EF0AF801EB5FFB4F882319F08081816075
:103F300002C080818E7F808380915A06C82FD0E096
:103F4000C7018C599F4F0E94EF0AC55BDB4F8883E6
:103F500080915A06C82FD0E0C7018A599F4F0E940E
:103F6000EF0A90E00E94A31CC35BDB4F88830091A3
:103F70005A0610E0C70182599F4F0E94EF0AF801CC
:103F8000EB5FFB4F882319F08081846002C0808141
:103F90008B7F808380915A06C82FD0E0C70180595B
:103FA0009F4F0E94EF0AC15BDB4F888380915A06C6
:103FB000C82FD0E0C7018E589F4F0E94EF0A90E0B3
:103FC0000E94A31CCF5ADB4F888300915A0610E051
:103FD000C70184579F4F0E94EF0AF801EB5FFB4F28
:103FE000882319F08081806802C080818F77808368
:103FF00080915A06C82FD0E0C70182579F4F0E9478
:10400000EF0ACD5ADB4F888380915A06C82FD0E043
:10401000C70180579F4F0E94EF0A90E00E94A31CA7
:10402000CB5ADB4F888300915A0610E0C7018E56A9
:104030009F4F0E94EF0AF801EB5FFB4F882319F0B6
:104040008081826002C080818D7F808380915A064A
:10405000C82FD0E0C7018C569F4F0E94EF0AC55A67
:10406000DB4F888380915A06C82FD0E0C7018A565B
:104070009F4F0E94EF0A90E00E94A31CC35ADB4F9F
:10408000888300915A0610E0C7018C589F4F0E9408
:10409000EF0AF801EB5FFB4F882319F080818860FD
:1040A00002C08081877F808380915A06C82FD0E02C
:1040B000C7018A589F4F0E94EF0AC95ADB4F888375
:1040C00080915A06C82FD0E0C70188589F4F0E94A0
:1040D000EF0A90E00E94A31CC75ADB4F888300912F
:1040E0005A0610E0C70186589F4F0E94EF0AF80158
:1040F000EB5FFB4F882319F08081806102C08081D3
:104100008F7E808380915A06C82FD0E0C7018458E3
:104110009F4F0E94EF0AC15ADB4F888380915A0655
:10412000C82FD0E0C70182589F4F0E94EF0A90E04D
:104130000E94A31CCF59DB4F888300915A0610E0E0
:10414000C70180589F4F0E94EF0AF801EB5FFB4FB9
:10415000882319F08081806202C080818F7D8083F6
:1041600080915A06C82FD0E0C7018E579F4F0E94FA
:10417000EF0ACD59DB4F888380915A06C82FD0E0D3
:10418000C7018C579F4F0E94EF0A90E00E94A31C2A
:10419000CB59DB4F888300915A0610E0C7018A573C
:1041A0009F4F0E94EF0AF801EB5FFB4F882319F045
:1041B0008081806402C080818F7B808380915A06D9
:1041C000C82FD0E0C70188579F4F0E94EF0AC959F6
:1041D000DB4F888380915A06C82FD0E0C7018657ED
:1041E0009F4F0E94EF0A90E00E94A31CC759DB4F2B
:1041F000888300915A0610E0C7018C559F4F0E949A
:10420000EF0AF801E95FFB4F882319F08081816094
:1042100002C080818E7F808380915A06C82FD0E0B3
:10422000C7018A559F4F0E94EF0AC559DB4F88830B
:1042300080915A06C82FD0E0C70188559F4F0E9431
:10424000EF0A90E00E94A31CC359DB4F88830091C2
:104250005A0610E0C70180559F4F0E94EF0AF801EF
:10426000E95FFB4F882319F08081846002C0808160
:104270008B7F808380915A06C82FD0E0C7018E546F
:104280009F4F0E94EF0AC159DB4F888380915A06E5
:10429000C82FD0E0C7018C549F4F0E94EF0A90E0D6
:1042A0000E94A31CCF58DB4F888300915A0610E070
:1042B000C7018A549F4F0E94EF0AF801E95FFB4F44
:1042C000882319F08081886002C08081877F808385
:1042D00080915A06C82FD0E0C70188549F4F0E9492
:1042E000EF0ACD58DB4F888380915A06C82FD0E063
:1042F000C70186549F4F0E94EF0A90E00E94A31CC2
:10430000CB58DB4F888300915A0610E0C7018454D4
:104310009F4F0E94EF0AF801E95FFB4F882319F0D5
:104320008081806102C080818F7E808380915A0667
:10433000C82FD0E0C70182549F4F0E94EF0AC9588E
:10434000DB4F888380915A06C82FD0E0C701805484
:104350009F4F0E94EF0A90E00E94A31CC758DB4FBA
:10436000888300915A0610E0C701845A9F4F0E942B
:10437000EF0AF801E95FFB4F882319F08081806420
:1043800002C080818F7B808380915A06C82FD0E045
:10439000C701825A9F4F0E94EF0AC558DB4F88839E
:1043A00080915A06C82FD0E0C701805A9F4F0E94C3
:1043B000EF0A90E00E94A31CC358DB4F8883009152
:1043C0005A0610E0C70180529F4F0E94EF0AF80181
:1043D000E75FFB4F882319F08081846002C08081F1
:1043E0008B7F808380915A06C82FD0E0C7018E5101
:1043F0009F4F0E94EF0AC158DB4F888380915A0675
:10440000C82FD0E0C7018C519F4F0E94EF0A90E067
:104410000E94A31CCF57DB4F888300915A0610E0FF
:10442000C7018C529F4F0E94EF0AF801E75FFB4FD4
:10443000882319F08081826002C080818D7F808313
:1044400080915A06C82FD0E0C7018A529F4F0E9420
:10445000EF0ACD57DB4F888380915A06C82FD0E0F2
:10446000C70188529F4F0E94EF0A90E00E94A31C50
:10447000CB57DB4F8883DF91CF911F910F91FF9036
:10448000EF9008954F925F927F928F929F92AF929A
:10449000BF92CF92DF92EF92FF920F931F93DF9321
:1044A000CF93CDB7DEB7C854D0400FB6F894DEBF77
:1044B0000FBECDBF04EA14E0C8010E949805C801F0
:1044C00066E049E00E947304C8010E944B0500D0D9
:1044D00000D0EDB7FEB71283018386E092E09483AB
:1044E00083830E946A2A0F900F900F900F90C8014B
:1044F0000E942F0500D000D007E814E0EDB7FEB70A
:104500001283018386EF91E0948383830E946A2A59
:104510005BEE452E51E0552EEE24FF24CC24DD2405
:104520000F900F900F900F90702E012F49E0A42E46
:10453000B12CAC0EBD1E4E010894811C911C87E865
:1045400094E00E941E2B982F8D3031F08D30DCF1DD
:1045500080538230C0F530C01830A1F59981892F81
:104560008053823078F5913311F490E801C090E0E7
:104570008A81813309F4905C8B81813309F4905EE8
:104580008C81813309F4905F8D81813309F4985FC8
:104590008E81813309F49C5F8F81813309F49E5FA2
:1045A0008885813309F49F5FF501EE0DFF1D90832F
:1045B0000894E11CF11C06C0F401E10FF11D908389
:1045C0001F5F01C010E0F0E4EF16F104C9F484EAC3
:1045D00094E0B601A5010E9483040894C11CD11C7B
:1045E00000D000D0EDB7FEB77182028354824382BF
:1045F0000E946A2AEE24FF240F900F900F900F90D4
:10460000FFEFCF16D10409F00CF499CFC85BDF4F50
:104610000FB6F894DEBF0FBECDBFCF91DF911F91D3
:104620000F91FF90EF90DF90CF90BF90AF909F9051
:104630008F907F905F904F900895DF92EF92FF925E
:104640000F931F93DF93CF93CDB7DEB72A970FB6A3
:10465000F894DEBF0FBECDBF73E0E72EF12CEC0E59
:10466000FD1E63E0D62E21C40E94143260527E44A7
:1046700080409040C8F40E941432695873418040D1
:10468000904090F01A3011F01D3031F480912306E3
:104690008F5F8093230602C0109223068091230629
:1046A000833011F40E944222812F69E175E00E945B
:1046B000F506882311F400E0F2C380911D05909166
:1046C0001E05A0911F05B0912005863E46EA94077D
:1046D00046E2A4074DE7B40709F4A0C2873E56EAB4
:1046E000950756E2A5075DE7B50708F0F8C08832E0
:1046F000EEE59E07E2EDAE07E4E2BE0709F439C23B
:104700008932FEE59F07F2EDAF07F4E2BF0708F03C
:1047100073C080352FED92072DEEA20728E1B20776
:1047200009F479C381353FED93073DEEA30738E1E6
:10473000B30788F584304AE9940747EDA4074EE0B3
:10474000B40709F416C285305AE9950757EDA50755
:104750005EE0B50780F48E3FEBEC9E07E7ECAE071A
:10476000E9E0BE0709F482C386519A4AA743BB40D9
:1047700009F08BC3FEC1823923EA92072CEEA2070F
:1047800024E1B20709F4F5C188599C42AA41B64117
:1047900009F07BC3F7C184344BED940740E7A407CD
:1047A0004DE1B40709F462C385345BED950750E72A
:1047B000A5075DE1B50780F48E3CE8E49E07E7E5D8
:1047C000AE07EAE1BE0709F429C284579B4EAA4707
:1047D000BB4109F05AC3CDC1823D22EC920722E8C9
:1047E000A2072EE1B20709F4CDC18C5A9A4CA64E0D
:1047F000B04209F04AC33AC3883546EB94074DEFFF
:10480000A4074AE4B40709F4E8C2893556EB9507D2
:104810005DEFA5075AE4B50788F5863EE5ED9E07EE
:10482000EAEDAE07E3E3BE0709F451C1873EF5EDBB
:104830009F07FAEDAF07F3E3BF0780F48E3729EA4D
:1048400092072BE5A20726E2B20709F49BC1825525
:104850009342A649B64209F018C36FC2883F4CEA9A
:1048600094074EEEA40744E3B40709F4FFC2865A46
:104870009E40A241B84409F008C398C28036EBEDCF
:104880009E07EBE3AE07EEE6BE0709F472C1813680
:10489000FBED9F07FBE3AF07FEE6BF0780F4823E18
:1048A00025E592072CE9A20726E6B20709F4A5C27E
:1048B0008C5E9943A647BB4609F0E7C2D7C28A3B44
:1048C00047EC940741E2A40744E7B40709F4FFC0AA
:1048D0008A57974CA94DBB4709F0D7C2C7C28C363F
:1048E000E8E69E07E3E4AE07E2ECBE0709F406C281
:1048F0008D36F8E69F07F3E4AF07F2ECBF0708F048
:1049000073C08A3726EF920721EFA2072DE9B2077D
:1049100009F484C18B3736EF930731EFA3073DE9E4
:10492000B30788F58C3845E8940747EAA40748E9B7
:10493000B40709F473C18D3855E8950757EAA50700
:1049400058E9B50780F48634E3E09E07E2ECAE0751
:10495000E5E8BE0709F491C282559A4EA048BA48CC
:1049600009F093C206C18A362EE2920722E6A20718
:1049700029E9B20709F41AC28E579241AA46BB49E7
:1049800009F083C2F6C08A3847EF940747ECA407C2
:1049900048EBB40709F4F6C08B3857EF950757EC8E
:1049A000A50758EBB50780F48E3FE6EB9E07E9E2DA
:1049B000AE07E5EABE0709F431C180529E44A94A18
:1049C000B14B09F062C219C2843A20E092072BE988
:1049D000A2072AEBB20709F449C28A5B9448A542B0
:1049E000BE4B09F052C209C2843649ED940740EE2D
:1049F000A40747EDB40709F46AC0853659ED950759
:104A000050EEA50757EDB50788F58435EDE29E0712
:104A1000EFEFAE07E5ECBE0709F4ABC08535FDE26C
:104A20009F07FFEFAF07F5ECBF0780F4803824E75E
:104A3000920720E1A20724ECB20709F4A3C086582C
:104A40009B43A04AB44C09F020C2D7C188324FE939
:104A5000940740E0A40747ECB40709F45FC1865906
:104A60009543A840B24D09F010C267C18E34EDE500
:104A70009E07EEE3AE07E3EEBE0709F47AC08F347B
:104A8000FDE59F07FEE3AF07F3EEBF0780F4843731
:104A900027E3920724EDA2072EEDB20709F4ADC17A
:104AA000865B9342A34AB24E09F0EFC1B7C0823988
:104AB00040E7940746E8A4074BEFB40709F4D6C1D2
:104AC000825F9D4EA442BD4F09F0DFC19FC10E948D
:104AD00014326093C8047093C9048093CA049093FD
:104AE000CB04D092C70489E195E060E170E00E94B8
:104AF000C9080E9441357093CD046093CC0489E1CC
:104B000095E064E170E00E94C9080E94413570930D
:104B1000CF046093CE0489E195E068E170E00E94E3
:104B2000C9080E9441358B017093D1046093D00471
:104B30006091D2047091D3048091D4049091D504F3
:104B400020E030E040E050E00E94D234882379F445
:104B5000B801882777FD8095982F0E94743560935F
:104B6000D6047093D7048093D8049093D90401E0BD
:104B70008DC1809123058093DA0480912405809370
:104B8000DB0483C189E195E060E070E00E94C90820
:104B900020E030E048EC52E40E94A7360E94413504
:104BA0007093DD046093DC04693C710520F0109281
:104BB000DD041092DC0480913D0590913E059093B8
:104BC000DF048093DE0480913F059091400590932F
:104BD000E1048093E0048091430590914405909313
:104BE000A4028093A3028091470590914805909379
:104BF000A6028093A5028091490590914A05909361
:104C0000A8028093A70280914B0590914C059A834E
:104C100089839093AA028093A90237C160912305EA
:104C20007091240580912505909126050E94743588
:104C300020E836E948E15BE40E94D9346093D2046D
:104C40007093D3048093D4049093D5046091270586
:104C5000709128058091290590912A05D7016C93C0
:104C600011967C93119712968C93129713969C939E
:104C70000E94743520E836E948E15BE40E94D934AB
:104C80006093E2047093E3048093E4049093E5045A
:104C9000809148058093E6048091470584300CF0AC
:104CA00083E08093E70489E195E060E170E00E9491
:104CB000C9086093D6047093D7048093D804909366
:104CC000D90489E195E068E070E00E94C90860932A
:104CD000E8047093E9048093EA049093EB0489E17B
:104CE00095E064E170E00E94C9086093EC04709361
:104CF000ED048093EE049093EF04C7C089E195E042
:104D000068E070E00E94C90890586093F0047093C6
:104D1000F1048093F2049093F304B7C089E195E025
:104D200060E070E00E94C9086093F4047093F50499
:104D30008093F6049093F704A8C089E195E060E0C1
:104D400070E00E94C9086093F8047093F90480939E
:104D5000FA049093FB0489E195E064E070E00E941E
:104D6000C90820E030E048EC52E40E94A7360E94D7
:104D700041357093FD046093FC0489E195E064E1A2
:104D800070E00E94C9080E9441357093FF0460934F
:104D9000FE0489E195E068E170E00E94C9080E9484
:104DA000413570930105609300056FC089E195E07E
:104DB00064E070E00E94C9080E944135882777FDB1
:104DC0008095982F0E9474356093020570930305B7
:104DD000809304059093050558C089E195E068E04B
:104DE00070E00E94C9080E944135709561957F4F1F
:104DF000709307056093060548C0809183058093F2
:104E0000080580918405809309053FC080912305A2
:104E100080930A053AC089E195E060E070E00E9465
:104E2000C90860930B0570930C0580930D05909352
:104E30000E0589E195E064E070E00E94C908609386
:104E40000F0570931005809311059093120589E169
:104E500095E068E070E00E94C908609313057093C4
:104E6000140580931505909316050FC080912F05AA
:104E7000809317058091340506C08091300580939A
:104E80001705809135058093180500E080911A057B
:104E9000823229F489E195E063E20E94E1098EEB18
:104EA00090E00E947B32002331F587E894E00E9475
:104EB000EE2A18161906F4F487E894E00E941E2BD7
:104EC000182F8091C704882309F0EECBCDCB109228
:104ED000C70401E0802F90E02A960FB6F894DEBF59
:104EE0000FBECDBFCF91DF911F910F91FF90EF903B
:104EF000DF90089500E02091C8043091C9044091EA
:104F0000CA045091CB04205F384D4F4F5F4F2F8321
:104F1000388749875A870E9414322F8138854985FE
:104F20005A85261737074807590788F2D3CFEF92DB
:104F3000FF920F931F9380915806882351F081E0D0
:104F40000E94B03364E070E00E94E137609328066D
:104F50003CC081E00E94B033AA2797FDA095BA2FEC
:104F6000BC01CD010E9474352DEC3CEC4CE45EE3B9
:104F70000E94A73620E030E040E85EE30E94A736BA
:104F80007B018C016091280670E0882777FD809571
:104F9000982F0E9474352DEC3CEC4CE45FE30E94AA
:104FA000A7369B01AC01C801B7010E940C340E94D6
:104FB000463520917306621730F030917206262F25
:104FC000361708F4232F209328061F910F91FF9086
:104FD000EF90089583E00E94AD3308951F93CF931F
:104FE000DF9385E090E06CE070E00E941C1668EEB4
:104FF00073E080E090E00E94223287E894E00E9413
:105000006B2BC0E0D0E010E0CE016DE171E00E94BA
:10501000E137892BA9F41F5E84EA94E0612F4CE00C
:105020000E94730484EA94E00E944B0584EA94E0B1
:105030006EEE0E947B0584EA94E00E942F051051D9
:1050400061E070E080E090E00E942232219687E0EB
:10505000C13DD807C9F6DF91CF911F91089586E031
:1050600061E00E94593308950F931F9386E061E039
:105070000E941A3307E814E0C80140E051EE60E0F6
:1050800070E00E948C2A1093A3060093A2060E944F
:105090002F2884EA94E00E94D1050E949A1C64EFB4
:1050A00071E080E090E00E94223283EF93E00E9462
:1050B000EF0A813011F00E94000D0E94600A1092E8
:1050C0005A0607C00E94B81C80915A068F5F8093D1
:1050D0005A0680915A068230A8F310925A060E940E
:1050E000EE270E94EA2786EB94E065E07AE224E668
:1050F00030E040E050E000E00E943F3184EA94E07C
:105100000E94980586EB94E00E94A5311F910F91B3
:1051100008952F923F924F925F926F927F928F925B
:105120009F92AF92BF92CF92DF92EF92FF920F9336
:105130001F93DF93CF9300D000D0CDB7DEB780911F
:105140005606882309F4E1C0E0907B06F0907C06C7
:1051500000917D0610917E06C801B7019F7725E377
:105160003AEF4EE85CE30E94A7360E94D63469838A
:105170007A838B839C83C801B7012091D20430913C
:10518000D3044091D4045091D5040E940B341B01E8
:105190002C019F7720EC3BE649ED57E40E94A736AF
:1051A0005B016C0160917F067091800680918106A1
:1051B000909182062091E2043091E3044091E4044E
:1051C0005091E5040E940B343B014C019F7720EC89
:1051D0003BE649ED57E40E94A73629813A814B818D
:1051E0005C810E94A7367B018C01C601B501A60136
:1051F00095010E94A7365B016C01C801B701A801A7
:1052000097010E94A7369B01AC01C601B5010E941F
:105210000C340E942E370E944135609349067093EA
:105220004A0680934B0690934C0660E070E080E85D
:105230009FE329813A814B815C810E94D9349B0193
:10524000AC01C201B1010E94A73697FA909497F879
:105250009094A40193010E947F3420EE3EE245E643
:1052600052E40E94A73620E030E044EB52E40E9472
:105270000C340E9441359B01AC0197FF04C02859B2
:105280003E4F4F4F5F4FCA01B901645B7040804091
:10529000904097FF06C0CA01B9016C547F4F8F4FF1
:1052A0009F4F0E9474352091D6043091D7044091CD
:1052B000D8045091D9040E940B340E94413597FFC5
:1052C00004C068597E4F8F4F9F4F0E94743520E075
:1052D00030E044EB53E40E94D93420E030E040E871
:1052E00051E40E94A7360E940A3720E030E040E8EF
:1052F0005FE30E940C340E9446356093480661319A
:1053000008F46CC01092480669C08091E7048230AE
:1053100008F464C08091E604853008F45FC0A09072
:1053200083068DE18A1508F459C0E090E804F090F6
:10533000E9040091EA041091EB04609184067091F5
:1053400085068091860690918706A80197010E94A4
:105350000B349F7720E030E040E05FE30E949C3612
:1053600018165CF410928306E0928406F09285068B
:10537000009386061093870631C08A2D8F5F809335
:1053800083068E3159F58091D2049091D304A09177
:10539000D404B091D50480937B0690937C06A093AF
:1053A0007D06B0937E068091E2049091E304A09183
:1053B000E404B091E50480937F0690938006A09367
:1053C0008106B0938206E0928806F09289060093E7
:1053D0008A0610938B0681E0809356060F900F90FB
:1053E0000F900F90CF91DF911F910F91FF90EF9051
:1053F000DF90CF90BF90AF909F908F907F906F90F5
:105400005F904F903F902F900895CF92DF92EF9250
:10541000FF920F931F930E94972780912806282FB1
:1054200030E03093AC022093AB0280915806882381
:1054300059F50091730610E0201B310BB901882744
:1054400077FD8095982F0E9474356B017C016091E7
:10545000720670E0601B710B882777FD8095982F8E
:105460000E9474359B01AC01C701B6010E94D9347A
:1054700020E030E048EC52E40E94A7360E9441351B
:105480007093AC026093AB0280910A058093AB02EB
:105490001092AC020E9452080E94F50A84EA94E03D
:1054A0000E9489280E94691A1F910F91FF90EF9026
:1054B000DF90CF9008950E941D23892B19F00E9440
:1054C000052A089586EB94E00E948D3108958FEFB0
:1054D0009FE70895DF93CF93CDB7DEB7FE013996EE
:1054E0008D819E8161E04F8158859F010E940B2D27
:1054F000CF91DF910895DF93CF93CDB7DEB7FE0153
:1055000039968D819E8160E04F8158859F010E9470
:105510000B2DCF91DF9108950F931F93DC01ED9137
:10552000FC910288F389E02D20E030E000E010E0FB
:1055300009951F910F9108958F92AF92CF92EF929C
:10554000FF920F931F93DF93CF93CDB7DEB7FC018C
:105550001382128288EE93E0A0E0B0E0848395830A
:10556000A683B7838AEE93E091838083558744872F
:1055700037872687118B008BF38AE28AC48AA58A33
:10558000868A70E0CB0123E0880F991F2A95E1F706
:105590009C012057394F308F278B8856994F928F17
:1055A000818F81E090E002C0880F991F6A95E2F731
:1055B0002091A006282B2093A006CF0140E051EEB9
:1055C00060E070E00E948C2ACF91DF911F910F91D3
:1055D000FF90EF90CF90AF908F900895FC01838D56
:1055E000882319F42FEF3FEF0DC00788F08DE02DD1
:1055F0002081318182819381281B390B848195819F
:1056000028233923C9010895FC01838D882319F4C7
:105610002FEF3FEF11C0018CF28DE02D2081318101
:1056200082819381281B390B209530958481958147
:10563000282339232F5F3F4FC9010895FC01838D33
:10564000882361F0A789B08D2D913C911197129616
:105650008D919C9113972817390721F44FEF5FEF35
:10566000CA01089512968D919C9113971696ED910B
:10567000FC911797E80FF91F408112968D919C912C
:105680001397019614962D913C911597822393239D
:1056900013969C938E93129750E0E2CFFC01838D7A
:1056A000882351F00788F08DE02D2081318182819F
:1056B00093812817390721F42FEF3FEFC90108958F
:1056C000828193810680F781E02DE80FF91F8081A8
:1056D000282F30E0F3CFDC015796ED91FC915897DD
:1056E00082819381918380835996ED91FC915A97A1
:1056F00080819181938382830895DC015B968C91F4
:105700005B978823A9F15996ED91FC915A972081D6
:1057100031812F5F3F4F84819581282339235C9607
:105720008C915C97882329F082819381281739070F
:10573000F9F08281938128173907D9F3808191810B
:105740000680F781E02DE80FF91F60835996ED91EF
:10575000FC915A97318320835296ED91FC91539797
:10576000808156969C91892B808321E030E002C095
:1057700020E030E0C9010895CF93DF93EC011B8254
:105780001A828A819B81998388831D821C828E81E3
:105790009F81009721F00E94C5031F821E82DF9126
:1057A000CF9108950F931F938C01DC015296ED91D8
:1057B000FC915397208156968C91569755969C91C3
:1057C0005597892B80958223808357968D919C9144
:1057D00058970E94BC2BF801818D928D0E94BC2BA2
:1057E000D8015B961C921F910F9108950F931F9300
:1057F000CF93DF938C01FC0113821282828193810B
:105800009183808341E0A1E0B0E001C04F5FFD01E2
:10581000042E02C0EE0FFF1F0A94E2F79B0182E004
:105820006130780710F020E032E0E217F30770F300
:10583000C1E0D0E002C0CC0FDD1F4A95E2F721970E
:10584000F801268137812115310541F08481958148
:105850008C179D0789F0C9010E94C503F801D58303
:10586000C483CE0101960E941B039C01F80197831B
:10587000868380E0232B09F081E0DF91CF911F9197
:105880000F910895AF92BF92CF92DF92EF92FF9265
:105890000F931F93CF93DF937C015A016B01E901B2
:1058A000DC015B968C915B978823F1F02115310523
:1058B00039F45796ED91FC915897C481D581219682
:1058C0000115110549F4D7015996ED91FC915A97AC
:1058D000048115810F5F1F4FD701ED91FC91008866
:1058E000F189E02DC7010995F7018789908D2097EF
:1058F00011F4C0E8D0E0BE010E94F62B882381F0AD
:10590000D70159968D919C915A970115110511F463
:1059100000E110E0B8010E94F62B882309F04DC089
:10592000D701ED91FC910088F189E02DC70109951F
:1059300067C0D7015096ED91FC915197B0E0AB163E
:10594000B1EEBB06B0E0CB06B0E0DB0609F454C014
:1059500081E090E0D70154960C9002C0880F991F07
:105960000A94E2F7808360E079E08DE390E0A6019D
:1059700095010E9416382150304040405040CA01E5
:10598000B90122E030E040E050E00E941638D70133
:105990001C96ED91FC911D9730831E96ED91FC9124
:1059A0001F972083D7015296ED91FC9153978081E8
:1059B00055969C91892B808323C0D7015996ED91F0
:1059C000FC915A9713821282828193819183808302
:1059D0005796ED91FC9158971382128282819381A0
:1059E0009183808381E05B968C931A141B041C04C2
:1059F0001D040CF49ECFD6CF108220E130E0C7CF3B
:105A0000DF91CF911F910F91FF90EF90DF90CF909A
:105A1000BF90AF9008952F923F924F925F926F92F6
:105A20007F928F929F92AF92BF92CF92DF92EF922E
:105A3000FF920F931F93DF93CF93CDB7DEB7649799
:105A40000FB6F894DEBF0FBECDBF3C01688B5A8BFA
:105A5000498B69011C01AE014F5F5F4F5C8B4B8B23
:105A6000E989FA89488940FD659140FF6191FA8B87
:105A7000E98B662309F4D7C3653249F440FD85916B
:105A800040FF8191FA8BE98B8532B1F40CC06A300A
:105A900051F4D301ED91FC910190F081E02DC10111
:105AA0006DE009956AE0D301ED91FC910190F081E0
:105AB000E02DC1010995D4CF982F10E088249924B6
:105AC0001032B0F49B3269F09C3228F4903251F0DD
:105AD000933271F40BC09D3239F0903349F4116068
:105AE00028C01260146025C0186023C0106121C056
:105AF00017FD2BC0892F80538A3078F416FF06C01B
:105B0000BAE09B9E902C1124980E13C0EAE08E9E62
:105B1000802C1124880E10620CC09E3221F416FDD8
:105B200082C3106406C09C3611F4106802C0983617
:105B300061F4E989FA89488940FD959140FF919186
:105B4000FA8BE98B992309F0BBCF892F85548330D9
:105B500020F4812F8061905E07C0892F85568330A5
:105B600008F0E6C1812F8F7E86FD02C076E0972E79
:105B70006FE3F62EF822953619F450E4F52A07C0A3
:105B8000963619F480E8F82A02C091109A94F7FE2C
:105B90000BC09BE3991520F427E05CE3B52E0DC004
:105BA000B92CB39427E009C0A7E0A91520F447E079
:105BB000942E27E001C0292DBB24F6013496FD87E1
:105BC000EC87D6016D917D918D919C91AE014F5FD7
:105BD0005F4F0B2D0E9443026C010981E02FF0E022
:105BE000FF87EE8700FF05C0FE85F3FD02C01DE2C2
:105BF00009C0F1FE02C01BE205C0F2FC02C010E0C9
:105C000001C010E28E859F858C709070892B09F4FD
:105C100044C0112311F483E001C084E0881510F022
:105C200088240EC0881AF3FC0BC0D301ED91FC91BF
:105C30000190F081E02DC10160E209958A94A9F7F5
:105C4000112349F0D301ED91FC910190F081E02DF9
:105C5000C101612F0995BE85B3FF03C00FE013E0BA
:105C600012C003E113E00FC0E114F10409F0605227
:105C7000D301ED91FC910190F081E02DC1010995D6
:105C80000F5F1F4F05C0EF2CFF24B0E1EB22FF2474
:105C9000F8016491662341F748C1F7FE13C0BC0CBC
:105CA000FE85F4FF04C08A81813309F4BA941B1481
:105CB0001CF0BB24B3942DC048E04B1550F538E0E0
:105CC000B32E27C0F6FC25C0892D90E08C159D05CC
:105CD0004CF05CEFC5165FEFD50624F080E8F82A9B
:105CE00001C09A94992049F0E2E0F0E0EC0FFD1F2A
:105CF000E90DF11D80818033A1F3F7FE0AC0B92CB4
:105D0000B394892D90E0C816D90614F0992401C0E7
:105D10009C18F7FC03C025E030E009C01C141D04EA
:105D20001CF021E030E003C096012F5F3F4F1123AC
:105D300011F02F5F3F4F992029F0892D90E00196B7
:105D4000280F391F882D90E02817390714F0882470
:105D500001C0821A4F2C5524C20189709070892B82
:105D600059F00CC0D301ED91FC910190F081E02D30
:105D7000C10160E209958A948820A1F7112349F0B6
:105D8000D301ED91FC910190F081E02DC101612FD3
:105D9000099543FE0BC00CC0D301ED91FC9101901D
:105DA000F081E02DC10160E309958A948820A1F774
:105DB000F7FE51C08601D7FE02C000E010E0760178
:105DC0000894E11CF11CE01AF10AE1E0F0E0EC0FAC
:105DD000FD1FEE0EFF1E26014B185108892D90E085
:105DE000AA24BB24A81AB90AFFEF0F3F1F0749F4E2
:105DF000D301ED91FC910190F081E02DC1016EE2A3
:105E00000995C016D10634F0401651061CF4F7016E
:105E1000608101C060E3015010400894E11CF11C56
:105E20000A151B054CF0D301ED91FC910190F08116
:105E3000E02DC1010995D8CF0C151D0541F48A81CB
:105E4000863320F4853319F4BE85B4FF61E3D301B2
:105E5000ED91FC9165C06A81613309F00F7ED30139
:105E6000ED91FC910190F081E02DC10109959920FF
:105E7000E1F0D301ED91FC910190F081E02DC101A1
:105E80006EE2099512E0E1E0F0E0EC0FFD1FE10F9A
:105E9000F11D60811F5FD301ED91FC910190F081B4
:105EA000E02DC10109959A9471F7D301ED91FC9110
:105EB0000190F081E02D44FC02C065E601C065E47C
:105EC000C1010995D7FC05C0C114D10441F404FFF8
:105ED00006C0D094C194D108D3946DE201C06BE2A6
:105EE000D301ED91FC910190F081E02DC101099564
:105EF00060E305C06F5FE6EFFFEFCE0EDF1EFAE056
:105F0000CF16D104BCF7D301ED91FC910190F08143
:105F1000E02DC1010995D301ED91FC916C2D605DDF
:105F20000190F081E02DC1010995CC84DD8478C118
:105F3000933631F0933799F0933509F061C023C05F
:105F4000F601808189835E010894A11CB11C42E0A6
:105F500050E0C40ED51E21E0E22EF12C12C0D60175
:105F6000AD90BC9016FD03C06FEF7FEF02C0692DAE
:105F700070E0E2E0F0E0CE0EDF1EC5010E942804D2
:105F80007C011F7713C0D601AD90BC9016FD03C0F5
:105F90006FEF7FEF02C0692D70E0E2E0F0E0CE0E1F
:105FA000DF1EC5010E941D047C01106813FF0BC099
:105FB00023C0D301ED91FC910190F081E02DC1014E
:105FC00060E209958A94882D90E0E816F90688F336
:105FD00013C0F50117FD659117FF61915F01D301B2
:105FE000ED91FC910190F081E02DC10109958110A6
:105FF0008A940894E108F108E114F10451F710C102
:10600000943611F0993699F517FF0AC0F6012081F0
:1060100031814281538184E090E0C80ED91E0CC0CA
:10602000D6018D919C919C01442737FD4095542FBA
:10603000E2E0F0E0CE0EDF1E9FE6F92EF12257FFE0
:1060400009C050954095309521953F4F4F4F5F4F78
:10605000F0E8FF2ACA01B901AE014F5F5F4F2AE0A5
:1060600030E00E94E501E82E4B89E41A41C09537E3
:1060700021F41F7E2AE030E01CC0197F9F3661F0BA
:10608000903720F4983509F0CEC00FC0903739F022
:10609000983709F0C8C004C028E030E00AC0106199
:1060A00014FD146020E130E004C014FD166020E10E
:1060B00032E017FF08C0D6016D917D918D919C91C2
:1060C000E4E0F0E008C0D6018D919C91BC0180E035
:1060D00090E0E2E0F0E0CE0EDF1EAE014F5F5F4FDA
:1060E0000E94E501E82EFB89EF1A8FE7F82EF122D6
:1060F000F6FE0BC04EEFF422E91438F4F4FE07C0AC
:10610000F2FC05C05FEEF52202C01E2D01C0192D64
:10611000F4FE0DC0FE01EE0DF11D8081803319F4F7
:1061200089EEF82208C01F5FF2FE05C003C08F2D64
:10613000867809F01F5F0F2DF3FC18C0F0FE13C026
:10614000181510F09E2C0FC09E2C980C911A182D2B
:106150000AC0D301ED91FC910190F081E02DC101C5
:1061600060E209951F5F1815A0F304C0181510F41C
:10617000811A01C0882404FF17C0D301ED91FC915E
:106180000190F081E02DC10160E3099502FF29C073
:10619000D301ED91FC910190F081E02D01FD02C051
:1061A00068E712C068E510C0802F8678D1F001FF43
:1061B00002C06BE201C060E2F7FC6DE2D301ED9139
:1061C000FC910190F081E02DC10109950AC0D30135
:1061D000ED91FC910190F081E02DC10160E3099502
:1061E0009A94E914A0F3EA94D301ED91FC91A1E013
:1061F000B0E0AC0FBD1FAE0DB11D0190F081E02DE0
:10620000C1016C910995EE2071F70AC0D301ED919F
:10621000FC910190F081E02DC10160E209958A9422
:106220008820A1F71DCC64960FB6F894DEBF0FBE90
:10623000CDBFCF91DF911F910F91FF90EF90DF9035
:10624000CF90BF90AF909F908F907F906F905F9016
:106250004F903F902F900895F999FECF72BD61BD88
:10626000F89A80B50895F999FECF1FBA72BD61BD45
:1062700040BD0FB6F894FA9AF99A0FBE08950F939D
:10628000FC016115710511F480E011C02183328396
:1062900043835483728761870170000F000F000FE2
:1062A0008081877F802B82608B7F808381E00F914C
:1062B0000895CF93DF93EC010E9414329B01AC014F
:1062C0008D819E81AF81B885281739074A075B0702
:1062D00028F4888184FD02C060E00DC089819A8124
:1062E000AB81BC81820F931FA41FB51F8D839E833A
:1062F000AF83B88761E0222757FD239533274427D2
:106300005527922F91709295907F88818F7E892B4F
:106310008883862FDF91CF910895CF93DF93EC018F
:10632000888182FF0FC0CE010E945931882351F02D
:10633000E985FA85309709F00995888183FF02C0C5
:106340008B7F8883DF91CF910895CF93DF93EC010A
:1063500089859A85892BE1F089819A81AB81BC81FD
:106360000097A105B105A1F00E94143229813A815C
:106370004B815C81260F371F481F591F2D833E8399
:106380004F835887888184608F7E888381E001C035
:1063900080E0DF91CF9108951F920F920FB60F9278
:1063A00011242F933F938F939F93AF93BF9380912B
:1063B000A8069091A906A091AA06B091AB063091CB
:1063C000AC060196A11DB11D232F2D5F2D3720F0A6
:1063D0002D570196A11DB11D2093AC068093A806F0
:1063E0009093A906A093AA06B093AB068091A40649
:1063F0009091A506A091A606B091A7060196A11DB1
:10640000B11D8093A4069093A506A093A606B09311
:10641000A706BF91AF919F918F913F912F910F90C0
:106420000FBE0F901F9018958FB7F8942091A80673
:106430003091A9064091AA065091AB068FBFB901D1
:10644000CA0108959B01AC017FB7F8948091A4061E
:106450009091A506A091A606B091A70666B5A89B47
:1064600005C06F3F19F00196A11DB11D7FBFBA2F66
:10647000A92F982F8827860F911DA11DB11D62E0BD
:10648000880F991FAA1FBB1F6A95D1F7BC012DC0A9
:10649000FFB7F8948091A4069091A506A091A60656
:1064A000B091A706E6B5A89B05C0EF3F19F001968D
:1064B000A11DB11DFFBFBA2FA92F982F88278E0FBE
:1064C000911DA11DB11DE2E0880F991FAA1FBB1FDE
:1064D000EA95D1F7861B970B885E9340C8F221504E
:1064E00030404040504068517C4F211531054105F6
:1064F000510571F60895019739F0880F991F880F9B
:10650000991F02970197F1F70895789484B58260F6
:1065100084BD84B5816084BD85B5826085BD85B547
:10652000816085BDEEE6F0E0808181608083E1E8F6
:10653000F0E010828081826080838081816080832E
:10654000E0E8F0E0808181608083E1EBF0E0808131
:1065500084608083E0EBF0E0808181608083EAE703
:10656000F0E080818460808380818260808380818C
:10657000816080838081806880831092C10008954B
:106580001F920F920FB60F9211242F933F934F93A8
:106590005F936F937F938F939F93AF93BF93EF938B
:1065A000FF938091AD069091AE06892B29F0E09182
:1065B000AD06F091AE060995FF91EF91BF91AF91B5
:1065C0009F918F917F916F915F914F913F912F910B
:1065D0000F900FBE0F901F9018951F920F920FB63D
:1065E0000F9211242F933F934F935F936F937F9359
:1065F0008F939F93AF93BF93EF93FF938091AF06D9
:106600009091B006892B29F0E091AF06F091B00689
:106610000995FF91EF91BF91AF919F918F917F91DC
:106620006F915F914F913F912F910F900FBE0F90FF
:106630001F901895CF93DF93482F50E0CA01875BD6
:106640009C4FFC0134914B5C5C4FFA018491882390
:1066500069F190E0880F991FFC01E95EFC4FA5915C
:10666000B491FC01EF5DFC4FC591D491662351F4C8
:106670002FB7F8948C91932F909589238C938881D0
:1066800089230BC0623061F42FB7F8948C91932F5B
:10669000909589238C938881832B88832FBF06C094
:1066A0009FB7F8948C91832B8C939FBFDF91CF91F0
:1066B0000895482F50E0CA01835A9C4FFC01249151
:1066C000CA01875B9C4FFC0194914B5C5C4FFA01C3
:1066D0003491332309F440C0222351F1233071F067
:1066E000243028F42130A1F0223011F514C02630D6
:1066F000B1F02730C1F02430D9F404C0809180007B
:106700008F7703C0809180008F7D8093800010C0C0
:1067100084B58F7702C084B58F7D84BD09C0809118
:10672000B0008F7703C08091B0008F7D8093B00060
:10673000E32FF0E0EE0FFF1FEF5DFC4FA591B4914A
:106740002FB7F894662321F48C919095892302C089
:106750008C91892B8C932FBF08958093AF0208955D
:10676000982F8E3008F09E5097708091AF028295DE
:10677000880F880F807C892B80937C0080917A0021
:10678000806480937A0080917A0086FDFCCF20910E
:10679000780040917900942F80E030E0282B392B4D
:1067A000C9010895CF92DF92EF92FF920F931F934A
:1067B000CF93DF937C016B018A01C0E0D0E00FC072
:1067C000D6016D916D01D701ED91FC910190F081A1
:1067D000E02DC7010995C80FD91F015010400115C0
:1067E000110571F7CE01DF91CF911F910F91FF90AD
:1067F000EF90DF90CF900895CF93DF930E94853282
:106800000E943428C0E0D0E00E945B2A2097E1F388
:106810000E940000F9CF5058BB27AA270ED041C2D2
:1068200001D230F006D220F031F49F3F11F41EF473
:10683000C0C10EF4E095E7FBB6C1E92F54D280F356
:10684000BA17620773078407950718F071F49EF56D
:106850006CC20EF4E0950B2EBA2FA02D0B01B901DE
:1068600090010C01CA01A0011124FF27591B99F0C6
:10687000593F50F4503E68F11A16F040A22F232FD2
:10688000342F4427585FF3CF469537952795A79522
:10689000F0405395C9F77EF41F16BA0B620B730BC9
:1068A000840BBAF09150A1F0FF0FBB1F661F771F3A
:1068B000881FC2F70EC0BA0F621F731F841F48F4EF
:1068C000879577956795B795F7959E3F08F0B3CF75
:1068D0009395880F08F09927EE0F9795879508955F
:1068E000A1D158F080E891E009F49EEFA2D128F000
:1068F00040E851E059F45EEF09C05BC116C2E92FD0
:10690000E078F1D168F3092E052AC1F3261737077D
:106910004807590738F00E2E07F8E02569F0E02502
:10692000E0640AC0EF6307F8009407FADB01B901DD
:106930009D01DC01CA01AD01EF934AD0B2D10AD06A
:106940005F91552331F02BED3FE049E450FD49ECD8
:1069500063CF0895DF93DD27B92FBF7740E85FE36A
:106960001616170648075B0710F4D92FE9D19F9335
:106970008F937F936F93BCD2E8E6F0E01DD191D165
:106980002F913F914F915F91EED1DD2349F09058C7
:10699000A2EA2AED3FE049EC5FE3D0785D274DDFC6
:1069A000DF917FC1DCD008F481E008954AD1E395FE
:1069B00089C10CD076C13DD140F034D130F021F402
:1069C0005F3F19F0F0C05111B1C1F3C08CD198F301
:1069D0009923C9F35523B1F3951B550BBB27AA2760
:1069E00062177307840738F09F5F5F4F220F331FD2
:1069F000441FAA1FA9F333D00E2E3AF0E0E830D09E
:106A000091505040E695001CCAF729D0FE2F27D0A0
:106A1000660F771F881FBB1F261737074807AB076E
:106A2000B0E809F0BB0B802DBF01FF2793585F4FE3
:106A30002AF09E3F510568F0B6C078C15F3FECF385
:106A4000983EDCF3869577956795B795F7959F5FA8
:106A5000C9F7880F911D9695879597F90895E1E0FC
:106A6000660F771F881FBB1F621773078407BA075B
:106A700020F0621B730B840BBA0BEE1F88F7E095B6
:106A8000089504D06894B11151C1089534D188F0AB
:106A90009F5790F0B92F9927B751A0F0D1F0660F0A
:106AA000771F881F991F1AF0BA95C9F712C0B13025
:106AB00081F03BD1B1E0089538C1672F782F882746
:106AC000B85F39F0B93FCCF3869577956795B39564
:106AD000D9F73EF490958095709561957F4F8F4FD3
:106AE0009F4F0895E89409C097FB3EF490958095D8
:106AF000709561957F4F8F4F9F4F9923A9F0F92F84
:106B000096E9BB279395F695879577956795B79501
:106B1000F111F8CFFAF4BB0F11F460FF1BC06F5FE7
:106B20007F4F8F4F9F4F16C0882311F096E911C0F9
:106B3000772321F09EE8872F762F05C0662371F01A
:106B400096E8862F70E060E02AF09A95660F771F2E
:106B5000881FDAF7880F9695879597F90895990F0A
:106B60000008550FAA0BE0E8FEEF16161706E80717
:106B7000F907C0F012161306E407F50798F0621B38
:106B8000730B840B950B39F40A2661F0232B242B0D
:106B9000252B21F408950A2609F4A140A6958FEF2C
:106BA000811D811D089597F99F6780E870E060E07E
:106BB00008959FEF80EC0895DF93CF931F930F9379
:106BC000FF92EF92DF927B018C01689405C0DA2E70
:106BD000EF01C9D0FE01E894A59125913591459129
:106BE0005591AEF3EF0129DEFE019701A801DA9479
:106BF00079F7DF90EF90FF900F911F91CF91DF9188
:106C000008959F938F937F936F93FF93EF939B01CF
:106C1000AC019DD0EF91FF91CFDF2F913F914F912C
:106C20005F9195C000240A941616170618060906E7
:106C3000089500240A9412161306140605060895F2
:106C4000B8CF59D0E8F3E894EFEFBB273FE048EC2A
:106C50005FE76B3D73078407950708F1FF279F5790
:106C6000B25A6A4D7F40894CF04032F4BE556542BD
:106C7000704F8643FF4F0894EE1F915030F0BB0FCA
:106C8000661F771F881FFF1FEBCF9EE7882332F018
:106C9000BB0F661F771F881F9A95C1F79395E095E4
:106CA00065C1092E0394000C11F4882352F0BB0F28
:106CB00040F4BF2B11F460FF04C06F5F7F4F8F4F14
:106CC0009F4F0895EF93E0FF06C0A2EA2AED3FE050
:106CD00049EC5FEBB2DDE5DF0F90039401FC9058C7
:106CE000E5E9F0E08ECF57FD9058440F551F59F05D
:106CF0005F3F71F04795880F97FB991F61F09F3FA9
:106D000079F087950895121613061406551FF2CFD1
:106D10004695F1DF08C0161617061806991FF1CF21
:106D200086957105610508940895E894BB27662748
:106D30007727CB0197F9089512DF08F48FEF0895B4
:106D40009B01AC0160E070E080E89FE332CE0BD0A5
:106D5000A8CF68DF28F06DDF18F0952309F023CF66
:106D600028CF1124E3CFBFDFA0F3959FD1F3950F78
:106D700050E0551F629FF001729FBB27F00DB11DBF
:106D8000639FAA27F00DB11DAA1F649F6627B00D4F
:106D9000A11D661F829F2227B00DA11D621F739F38
:106DA000B00DA11D621F839FA00D611D221F749F46
:106DB0003327A00D611D231F849F600D211D822F8D
:106DC000762F6A2F11249F5750408AF0E1F08823D4
:106DD0004AF0EE0FFF1FBB1F661F771F881F9150E1
:106DE0005040A9F79E3F510570F0DDCE9FCF5F3F29
:106DF000ECF3983EDCF3869577956795B795F79514
:106E0000E7959F5FC1F7FE2B880F911D969587959B
:106E100097F9089570DFE0F09E37D8F09639B8F40E
:106E20009E3848F4672F782F8827985FF9CF86958A
:106E30007795679593959539D0F3B62FB1706B0F11
:106E4000711D811D20F4879577956795939573C083
:106E50008DC06CCF11F40EF4ACCE88C04CDFD0F3F3
:106E60009923D9F3CEF39F57550B87FF8FD05695B3
:106E70009795B0E020F4660F771F881FBB1F1F9304
:106E80000F9300249001A0018001F001A0E80E0FF3
:106E90001F1F0A1E511D601B710B8009B50B48F4A2
:106EA000600F711F801DB51F0E1B1F0B0A0A5109B1
:106EB00007C02E0F3F1F4A1F0E0F1F1F0A1E511D16
:106EC000660F771F881FBB1FA695F795E795F8F605
:106ED0000617170708065B07211D311D411D0F917D
:106EE0001F91B901842F9158880F96958795089521
:106EF0009B01AC012CCFDF93D92FA3DEE695D7956C
:106F00002AED3FE049E45FE3B33A62077307840781
:106F10009507D7952AF0A2EA49EC90688EDCC1DE8D
:106F2000E3EBF0E06EDEDD0F0BF00ADFDD0F0BF4BC
:106F30009058DF910895882371F4772321F09850B9
:106F4000872B762F07C0662311F499270DC0905127
:106F5000862B70E060E02AF09A95660F771F881FF5
:106F6000DAF7880F9695879597F908959F3F49F02E
:106F7000915028F4869577956795B7959F5F8038EF
:106F80009F4F880F9695879597F908959150504097
:106F9000660F771F881FD2F70895AA1BBB1B51E10C
:106FA00007C0AA1FBB1FA617B70710F0A61BB70B79
:106FB000881F991F5A95A9F780959095BC01CD011E
:106FC000089597FB092E07260AD077FD04D0E5DF48
:106FD00006D000201AF4709561957F4F0895F6F75A
:106FE000909581959F4F0895A1E21A2EAA1BBB1B75
:106FF000FD010DC0AA1FBB1FEE1FFF1FA217B30785
:10700000E407F50720F0A21BB30BE40BF50B661F9A
:10701000771F881F991F1A9469F76095709580955E
:1070200090959B01AC01BD01CF01089597FB092EFE
:1070300005260ED057FD04D0D7DF0AD0001C38F447
:1070400050954095309521953F4F4F4F5F4F089594
:10705000F6F790958095709561957F4F8F4F9F4F74
:107060000895EE0FFF1F0590F491E02D0994F89418
:02707000FFCF50
:107072002563002563256300256325326925632581
:107082003032697C256325326925632530326900F7
:1070920025632532692563253032690025352E3076
:1070A20066256300256325312E3566256300256339
:1070B200253569256300256325352E326625630053
:1070C2006D616E0073743100737432007374330037
:1070D2007374340073743500737436007068200062
:1070E200636C200076722000686C200061702000C2
:1070F200727462006C616E0070702000706F6900C3
:1071020061632000006174200025632573002563FC
:1071120025332E30692563002534692563256300F4
:10712200256325336925630025737C256325732533
:10713200630020C0C0C0C0C0C7C0C0C0C0C0200063
:1071420025342E3066256300256325332E306625CF
:107152006300256325352E306625630025632531BE
:10716200312E36667C25632531312E366600256345
:107172002532690025332E31662563002020202028
:1071820020202020202020200020206469736172AA
:107192006D6564202000206E6F2074656C20636F23
:1071A2006D2000206E6F2067707320666978200062
:1071B20062617474207761726E696E6700626174D5
:1071C20074637269746963616C0020626174742013
:1071D2006572726F7220006C696E6B207175616CE2
:1071E200697479006D6167207761726E696E6700FC
:1071F2006D616720637269746963616C00206D61FF
:107202006720206572726F7220002573002000B51E
:10721200060000E803E803E803E8039DFF016401B8
:10722200000000007B05D23379047C047F048204D1
:10723200672A00070E091C1B1215383F363124231A
:107242002A2D70777E796C6B6265484F46415453A4
:107252005A5DE0E7EEE9FCFBF2F5D8DFD6D1C4C314
:10726200CACD90979E998C8B8285A8AFA6A1B4B304
:10727200BABDC7C0C9CEDBDCD5D2FFF8F1F6E3E474
:10728200EDEAB7B0B9BEABACA5A28F888186939464
:107292009D9A2720292E3B3C35321F1811160304D4
:1072A2000D0A5750595E4B4C45426F6861667374C4
:1072B2007D7A898E878095929B9CB1B6BFB8ADAA24
:1072C200A3A4F9FEF7F0E5E2EBECC1C6CFC8DDDA24
:1072D200D3D4696E676075727B7C51565F584D4A94
:1072E2004344191E171005020B0C21262F283D3A84
:1072F20033344E49404752555C5B7671787F6A6DF4
:1073020064633E39303722252C2B0601080F1A1DE3
:107312001413AEA9A0A7B2B5BCBB9691989F8A8D53
:107322008483DED9D0D7C2C5CCCBE6E1E8EFFAFD43
:10733200F4F3C2C0C0C1C0C0C1C0C0C4C0C0C1C0DB
:10734200C0C1C0C0C3C0C0C1C0C0C1C0C0C5C0C030
:10735200C1C0C0C1C0C0000000007D2BD233EE2AE4
:0E7362001E2B4E2B6B2B042B8C2AD22B422C75
:00000001FF
